:1020000000800020AD5F0000955F0000955F00003C
:1020100000000000000000000000000000000000C0
:10202000000000000000000000000000955F0000BC
:102030000000000000000000955F0000016000004B
:10204000955F0000955F0000955F0000955F0000C0
:10205000955F0000955F0000955F0000995F0000AC
:10206000955F0000F53C0000955F0000955F000063
:1020700015280000955F0000053D0000955F0000F9
:10208000955F0000955F0000955F0000955F000080
:1020900000000000955F0000955F0000955F000064
:1020A000955F0000955F0000955F0000955F000060
:1020B0000000000010B5064C2378002B07D1054B1B
:1020C000002B02D0044800E000BF0123237010BDA4
:1020D000300200200000000038C10000044B10B5A1
:1020E000002B03D00349044800E000BF10BDC046E8
:1020F000000000003402002038C1000010B5294C57
:1021000086B0200001F072FA274B200063610121A4
:1021100000F08FFF00232361244B0A2219686846D0
:1021200003F0CAFE694603A803F0E8FE204903A8AD
:1021300003F022FF0100200003F0E5FD03A803F0F7
:1021400060FE684603F05DFE2000012100F071FF93
:1021500080231B032361174B186806F0D7FB02008E
:102160000B006846144907F063FA6946200003F043
:10217000D1FD2000022100F05CFF1E2323610F4BE4
:10218000186806F0C3FB02000B0003A80C4907F017
:102190004FFA03A9200003F0BDFD200001F0FAFC76
:1021A00006B010BD4C020020010001000400002018
:1021B00044AD00000C00002046AD000008000020E7
:1021C0004CAD000070B5244800F008F9002815D186
:1021D0002249234803F0BAFD224C234D206806F023
:1021E00095FB224A224B04F02DFE06F0E1FB291C50
:1021F000061C04F057FD002827D126601D4800F07A
:10220000EDF8002815D11C49154803F09FFD154C29
:102210001A4D206806F07AFB144A154B05F0AAFF08
:1022200006F0C6FB291C061C04F028FD00280ED170
:102230002660134800F0CCF800280AD1FF211230A4
:1022400004F012F9FFF75AFF70BD2560D6E725604C
:10225000EFE700211220F3E7E802002052AD000072
:102260001C0A0020080000200000A0419A999999BA
:102270009999B93FD002002057AD00000000A0405E
:10228000B80200201FB532220621104800F066F87F
:10229000322207210E4800F061F8322211210D4848
:1022A00000F05CF80C4B0D4C02930D4B1022019387
:1022B00001235B42009360210A4B200001F07EF86D
:1022C000094A0A49200004F0F7FA1FBDE80200207D
:1022D000D0020020B8020020A08601004C0200209D
:1022E000801A0600000300200000002021340000B6
:1022F00037B5E121154D4902280002F063F8144971
:10230000280003F023FD0121122004F097F9002199
:10231000122004F0A9F801230E4C00933C22022164
:10232000200001F075F9002803D10B49280003F0C3
:1023300003FD200001F05AF9FA20400003F0A4FE4A
:102340000221200000F0F5FB37BDC0461C0A00202A
:102350005DAD00004C0200206DAD000070B50400C2
:102360000D00C8B20221160004F068F901232361B0
:10237000E3600023256066602000636170BD00009B
:10238000036870B50400D8B204F0D0F923690500E1
:10239000834202D003F042FE606103F03FFE6369B6
:1023A000C01A636898420ED9A368AB420BD0074E9F
:1023B0000A222168300003F016FD0A22A1683000CD
:1023C00003F015FDA560256170BDC0461C0A002004
:1023D00010B50400FFF7D4FFA06810BD10B50400CD
:1023E000FFF7CEFFA068E368984201D0E06010BD1F
:1023F00001204042FBE70020704710B503689C6B4A
:102400000123A04710BD8C2300229B00C154103B28
:10241000C3185A609A60DA6001238375704710B55B
:10242000036801211B6B984710BDF8B505000E002D
:1024300017000024BC4208D02B68315D1B682800BF
:102440009847002801D00134F4E72000F8BDFC30A3
:10245000406A704770478E239B00C15070478D23A0
:102460009B00C15070470300FC335A6A002A03D016
:102470001B6AC018007E704701204042FBE7000045
:1024800070B5060018250C49006901F033FF30696A
:1024900001F071FD2B000821307D084C4343E31807
:1024A000595604F05BF90821707D45436419615663
:1024B00004F054F970BDC046A0860100A4B8000025
:1024C00070B504000D00006901F06AFD2900206963
:1024D00001F010FF206901F04EFD70BD10B50069DC
:1024E00001F05EFD10BD0000F7B50193FA238026D0
:1024F000002504009B008360134B760008330F0017
:1025000045602900009203603200183006F066FB37
:1025100023002000FC332530DD6132001D622900DC
:102520005D62FF3006F05AFB88239B00E3185D6074
:102530009D60DD606B461B78276123756B461B79B8
:10254000A57520006375FEBD9CAD000070B506004A
:102550001825006901F0A9FE306901F00CFD2B007F
:102560000821307D064C4343E318595604F0F6F831
:102570000821707D45436419615604F0EFF870BD81
:10258000A4B8000010B50022FFF7E0FF10BD030063
:10259000802210B5FC33DC685200944208D05A689F
:1025A00081545A680132D2B25A60DA680132DA6074
:1025B00010BDF7B50400171E019302D100252800B5
:1025C000FEBD03000022FC33DA611A625A62006920
:1025D000013201F017FD061EF0D0230020691833E8
:1025E000009301F0A2FD01000098FFF7D0FF012544
:1025F0002069BD4214D001F076FD00280FD020697B
:1026000001F0E0FC0221206901F0E6FC206901F004
:102610008CFD01000098FFF7BAFF0135E8E70600DE
:10262000206901F0C7FC019B002B06D0002E06D0CC
:102630000321206901F0D0FCC1E7002EBFD1013D8C
:10264000BDE7002310B5827D9A420CD0882292000B
:102650008218D46880225200944204D02530FF3082
:10266000FFF795FF0123180010BD0300FC33DA6863
:10267000002A09D09A68805C9A680132D2B29A60C6
:10268000DA68013ADA60704701204042FBE7002235
:102690008C2370B59B00827504000E00C15C00693C
:1026A00001F0B0FC002806D10321206901F094FC60
:1026B0000225280070BD88239B00E318DD68002DEB
:1026C00011D020002530FF302569FFF7CEFFC1B2C1
:1026D000280001F0D9FC0028EDD10321206901F088
:1026E0007BFC0325E5E7002EE3D00321206901F000
:1026F00073FCDEE710B51830FFF7B7FF10BD70B5FB
:102700000400006901F0E6FC002815D0206901F002
:10271000F8FC002811D0206901F054FC0321206945
:1027200001F05AFC8E239B00E558002D35D1002383
:10273000FC34E3612362636270BD206901F0EBFC4D
:10274000002809D0206901F0E1FC002804D02069AC
:1027500001F0E6FC0028DED0206901F0DCFC002856
:1027600021D1206901F0C8FC0028E5D0206901F0E2
:10277000D7FC002833D088239B00E318DB68FF21B7
:10278000002B05D020002530FF30FFF76EFFC1B2CF
:10279000206901F091FCA075CEE7236820001B6939
:1027A0009847A847C3E7206901F00CFC2069032182
:1027B00001F012FC206901F0B3FC0028BCD0882392
:1027C00000229B00E3185A609A60DA600123A37527
:1027D0008D239B00E3589342AED09847ACE723008B
:1027E000FC335A6A802320695B009A4206D101F0CB
:1027F000E1FB0321206901F0EFFB9DE701F095FC6F
:10280000010020001830FFF7C2FE206901F0DAFB5A
:10281000EFE7000010B50248FFF771FF10BDC0469A
:102820000003002010B51523142202490248FFF7C7
:102830005BFE10BD040A0020000300207047F0B5C5
:102840001D0089B00EAB00241C5F0FAB1B88160067
:102850000693A31ADA179B18534002936B1ADA17E0
:102860009B1853400393039A029B0190934205DC0B
:1028700023002C001D0033000E001900A64205DCC9
:102880002B000D001900230034001E00331B9BB2E7
:1028900004934B1BDA179B18534007936B46102287
:1028A0009A5ED30F9B185B10009301238D4221DAAF
:1028B0000593B44224DC019B039A1B689B691F00AB
:1028C000029B934218DD22002900069B0198B8471D
:1028D000009B079A9B1A9BB21AB20092002A06DA52
:1028E000059AAD18049A2DB2D3181BB20093013487
:1028F00024B2DEE75B42DBE7069B2A002100E5E726
:1029000009B0F0BD704710B504682469A04710BD38
:1029100037B506AC258804680095A46BA04737BD81
:1029200037B506AC258804680095E46BA04737BD31
:1029300073B506AC0025655F07AC26880468019670
:102940000095246CA04773BDF0B5160004000D007F
:1029500085B003930AAB1F8803685B699847039BA4
:102960002268013B9B191BB200930197976A2B00C9
:10297000320029002000B84723682000DB6A98470E
:1029800005B0F0BDF0B505001C000E00170085B0C5
:102990000AAB1B88013C03930368A4195B69984741
:1029A00003992A680191009723B23100946A2800A4
:1029B0003A00A0472B682800DB6A984705B0F0BDB5
:1029C000F0B50E0087B003930CAB029200229B5E21
:1029D000050004930DAB1B883400059303685B6905
:1029E0009847039A2B68B21894420ADA059A210094
:1029F00000921F6A029A049B28000134B84724B24F
:102A0000EFE7DB6A2800984707B0F0BD13B50191E6
:102A10000E24015F0C22835E02680091146C002278
:102A20001100A04713BDF0B5040015000E0087B0DB
:102A300004930CAB00229B5E05930DAB1B880393A4
:102A400003685B699847039A236800925F6A2A00CB
:102A5000049B31002000B847059B03995A1E236848
:102A6000009152195F6A3100049B200012B2B847EE
:102A7000039A236800921F6A2A00059B31002000F8
:102A8000B8470499039A236801390092891909B259
:102A90001F6A2A00059B2000B84723682000DB6AD4
:102AA000984707B0F0BD7047F0B585B01E000AAB7F
:102AB0000027DF5F0BAB1B88140005000291039316
:102AC0000268B14210D1BC4202DC3B0027001C006E
:102AD000039901340091E31B966B1BB23A000299F3
:102AE0002800B04705B0F0BDBC4211D1029BB342F3
:102AF00002DC3300029E0293029B03990133009192
:102B00009B1BD76B1BB2220031002800B847E9E7B6
:102B100053699847039A2B68019200979F6A28008F
:102B2000330022000299B8472B682800DB6A9847D7
:102B3000D8E70323194010B50822835E81760A2462
:102B4000025F012904D0032902D08381C28110BD14
:102B50008281C381FBE700004281C281012252428F
:102B600042610222002310B5FF32074C0283013A72
:102B70000834FF3A436004600181818103618376F8
:102B8000C2760377036210BDECB20000F0B58DB0E1
:102B9000089312AB039200229B5E0791049313AB40
:102BA00000229B5E0400099314AB1B880A93036800
:102BB0005B6998470722049B039FD91DCB171340DD
:102BC0005B18DB10059300231D0001930B92039A01
:102BD000BBB206939B1A099A1BB29A422BDD0023C3
:102BE000049A93421EDA9AB202920B9A6D0099B23D
:102BF000EDB2114204D1089A0199DB105218D55C4C
:102C00006BB2002B0ADA079B029A2000D1182368C6
:102C100009B29B693A001E000A9BB047029E01362A
:102C200033B2DDE7059A019B9446069F6344013762
:102C300001933FB2CBE723682000DB6A98470DB0D1
:102C4000F0BD0000F0B595B01D001AAB1B88040064
:102C500005931BAB1E881CAB1B78089103931DAB1F
:102C60001B7804920293036A002B00D0C4E00C226C
:102C7000835E8B4200DC7DE00E22835E049A9342E9
:102C800078DD0623039A53435B18002B72DD029B09
:102C9000049ADB009B18002B6CDD037F002B03D113
:102CA000AF2D01D90135EDB2236820005B6998474B
:102CB00005235D430B9300230793984B5B190F93F8
:102CC000079A0F9B9B5C0A936B469B8B09936B4601
:102CD0009B890D936B460D9A1F8C099B5343FB18E0
:102CE0001BB20E9308230C930023069301220A9B28
:102CF0002068134252D06B461A8B198A039B012B12
:102D00003AD1029B012B37D1099B52188569D919F9
:102D1000059B12B209B22000A847069B01335BB2A3
:102D200006930A9B5B080A930C9B013BDBB20C9356
:102D3000002BDBD1079B01335BB207930B9B013B5D
:102D4000DBB20B93002BBBD1059BB3420ED0039B90
:102D50002268012B3FD1029B012B3CD10537009605
:102D6000156A39B20733049A2000A8472368200067
:102D7000DB6A984715B0F0BD6B460C255B5F029D82
:102D80006A438A18059912B2019169460825495F7C
:102D90000091C5690E992000A847BEE7059BB34284
:102DA000BBD06B46198B1A8A039B012B0AD1029B5D
:102DB000012B07D1099B5218D91912B209B28569A2
:102DC0003300A8E76B460C255B5F029D01966943C3
:102DD000521812B2D9E76B460C215B5E05210D98A3
:102DE0000196414302987918C0000090D56909B254
:102DF000049A2000A847B9E71A7AAD1AEDB25A68CA
:102E0000ED001B68551913932B880993AB780D932C
:102E1000EB7811930523EB560E930623EB560F9395
:102E2000039B012B02D8029B012B56D96B463822FB
:102E30009B5E0B936B463C229B5E0C9300272368A2
:102E400020005B69984707970697119B069A9A425C
:102E500000D38BE76B461B8A00260A930C9B9B18BA
:102E6000029A53430A9AD3181BB210933B000D9A4F
:102E700096424BD25A1CD2B212920722134207D169
:102E8000099B0999139A0133525C9BB207920993EB
:102E90006B461B7F5BB2002B17DA6B46198C039BCA
:102EA0002068012B1DD1029B012B1AD10A9B0F9A7E
:102EB0009A18069BD2180E9B12B2C91883698919F9
:102EC0001D0009B2059B2000A847079B01365B0047
:102ED000DBB20793F6B2129BC9E700230C930B9366
:102EE000ACE76B460C229B5E0B9A039D92196A43DA
:102EF0008918059A09B201926A460825525F009224
:102F0000C26920001500109AA847DEE7069D0D9BB8
:102F10000135FF18EBB2FFB2069396E7ECAD000067
:102F2000F0B5026A85B004000B00002A34D10A29EA
:102F300008D1437E0282DB00628A9B1863820120F3
:102F400005B0F0BD0D29FAD0E17E007E657E002936
:102F50000ED01026A15F0626464389190C27E65F8E
:102F6000B14205DD1226A15F2282EA005218628278
:102F70000290E08A1221625E0190A08A1026A15F71
:102F8000009003952000FFF75DFE0622237E534349
:102F9000228A9B182382D2E70A2905D100230382C3
:102FA000127B437E5343C7E70D29C8D0117A8B4269
:102FB000C5D3907A9842C2D3591AC9B25068C90091
:102FC0004518AF78002F28D0E978002925D0E17E78
:102FD000207E667E002913D005216956C919414318
:102FE0008C461021675EBC440C21675EBC4507DD42
:102FF0001227E15F00272782127B724352186282F8
:103000000290E08A1221625E0190A08A1027E15F9F
:10301000009003962000FFF715FE2B79227EB6E77D
:10302000002900D101310176002A00D10132427617
:10303000704710B50A00FFF7F3FF10BD70B506002A
:103040000C008D18AC4207D0336821789B683000A3
:10305000984720700134F5E770BD7047704710B590
:103060000400406800F048FF0023237610BD10B52F
:10307000406800F066FF10BDF8B5050040680C0020
:1030800000F05AFF2B68E7B2260A9B68012810D18E
:1030900039002800FF2798472B68BC4304439B68EE
:1030A000310028009847030220003840184380B2BE
:1030B000F8BD310028009847FF262B6800023440F5
:1030C00004439B68390028009847B4432043EEE747
:1030D00010B5040003F060F8200010BD10B54B1CC3
:1030E0000BD0102909D0EFF3108472B6102905DD3A
:1030F00002234376002C00D162B610BD0123427E2C
:103100001A43427618224A430449891816228A56DD
:103110009340C2691343C361ECE7C046A4B8000002
:103120004B1C17D0102915D0437E9B0712D4EFF308
:10313000108272B618234B430749C9180123897DB1
:1031400049B28B40C1699943C16100D14176002ADF
:1031500000D162B67047C046A4B80000437E002B81
:1031600005D09A0704D5837E002B00D062B6704745
:10317000DB07FCD5C369024A9BB2D360F7E7C046C0
:1031800000180040037E002B04D143768376C36190
:1031900001330376704700007FB5036902AE040077
:1031A0000D00029172608B4203D1828AB3889A42E9
:1031B00026D0200006223100103005F0F3FC6068B4
:1031C00000F0B1FE7379E17A013B581E8341227B06
:1031D00000936068002301F043F833790021013B3C
:1031E000DBB2022B01D8074AD15C074B2A009D4273
:1031F00000D91A00606800F067FE606800F089FE80
:103200007FBDC04644B30000001BB70070B5182650
:103210000400FFF7B7FF33000821207A0D4D434328
:10322000EB18595603F09AFA33000821A07A434369
:10323000EB18595603F092FA0821607A4643AD190B
:10324000695603F08BFA044B200006CBFFF7A4FF6E
:1032500070BDC046A4B800005C05002007B5437EE1
:1032600000910192002B07D09A070AD5EFF3108343
:103270005A425341837672B60099019AFFF78CFF48
:1032800007BDDB07F8D5C369014A9BB29360F3E73A
:10329000001800400E490F4B10B501220B600023AF
:1032A0004A710B710C490D48083101600C49427597
:1032B00041600C49C272018118210361817203755A
:1032C000094A0A490376037303F0F6FA10BDC046B3
:1032D0005C05002000093D0048B300003C050020CB
:1032E0000C0A002016170000000000205D300000CE
:1032F000F0B500291BDB0C25445F8C4217DD002A4A
:1033000015DB0E25445F944211DD847E022C0FD024
:10331000032C16D0012C04D1D2430489A4180A002E
:1033200021B2012B13D0002B22D0022B32D0F0BDC2
:103330000489013C611AD443428909B2121912B2BC
:10334000EFE74489013C641A110022B2E9E707253E
:10335000D4172C40A4182A4093400827C65FE410D5
:1033600074436118C46A61180A7813430B70DEE76E
:103370000724D31723409B180826855FDB106B4377
:103380005918C36A22405918012393401A000B7838
:103390009343EBE70724D31723400826855F9B1848
:1033A000DB106B435918C36A012022409040020091
:1033B00059180B785A400A70B9E7000070B500251B
:1033C00004001E0012B204AB09B25D57FFF7C4FB44
:1033D000104B08332360002363629E4200D10E4EDF
:1033E0002100FF223331A662E3620A704A708A70BC
:1033F000CA70220037321570059A2000A265069A1D
:10340000E265064A62662200643213710123537139
:1034100070BDC04624B800000003002000093D0034
:10342000054B10B5083304000360C06A002801D0C2
:1034300005F09CFB200010BD24B80000F8B5040086
:10344000806A0D00002814D02300303319780368F7
:10345000DB6A9847A06A002103681B689847A06A46
:10346000290003681B689847A06A03685B6B98474C
:10347000F8BD226C216D1368606A8B4313600028CD
:1034800004D0036829009B689847F1E70821802051
:10349000E36BA26BA76C166828420ED03E43166001
:1034A0001E68E76C01393E431E601E68E76C4008E9
:1034B000BE431E600029EDD1DAE7BE43EFE770B5E9
:1034C0000400806A0D00002812D00368A16D9B6A79
:1034D000984729004D1EA9412000A631FFF7AEFFF5
:1034E000A06A002812D00368E16D9B6A984770BDFE
:1034F000606A002804D00368616EDB69A26E984799
:10350000626C616D13688B431360E2E7626C616DFE
:103510001368606A0B4313600028E8D003681B6AD5
:103520009847E4E7F7B50400806A8B180D00019313
:1035300000282BD02700036830373978DB6A98479A
:10354000A06A0021036801261B689847A06A019AB7
:103550000368954217D0FE2E0CD95B6B9847A06A82
:10356000397803680126DB6A9847A06A002103685E
:103570001B689847A06A2978036801361B6898473A
:10358000B6B20135E2E75B6B9847F7BD226C216D5F
:1035900013688B431360019BAB42F6D02B78606AB3
:1035A0000093002805D0036800999B68984701356F
:1035B000F1E708208026E36BA26BA76C0099BC465C
:1035C00017680E420FD061460F4317601F68E16C09
:1035D00001380F431F601F68E16C76088F431F603E
:1035E0000028EAD1E3E761468F43EEE7072110B5F3
:1035F0000A22835E0733DA170A40D2180821435E95
:10360000D2105A43C06A002105F0E8FA10BD00004C
:10361000F0B587B004930CAB1B7804000593C36A24
:103620000E001500002B1BD02000FFF7DFFF0A2340
:10363000E25E0823E15E202A25DC203AD30F9A18A7
:103640000B00733BD90FC918012302931F3352108B
:10365000491001935333009312B209B2B04B24E0E6
:103660000A22835E07220733D8171040C0180822A9
:10367000A35EC010584305F06FFAE062031ED3D179
:10368000180007B0F0BD403AD30F9A180B00523B18
:10369000D90FC918012302933F33019312335210FB
:1036A000491000939F4B12B209B22000FFF76EFA47
:1036B000230031331E70A06A002800D19CE0002D49
:1036C00000D097E00A23E55E203D6B1E9D413C350E
:1036D000230030331D70059B002B00D11BE10368D4
:1036E000DB699847049B002B1BD025000020373551
:1036F0002856002815DBC0B2012102F09FFF0121EE
:10370000287802F0E7FF012002F0BEFC00212878B3
:1037100002F0E0FF0A2002F0B7FC2878012102F055
:10372000D9FFA06A002800D1CBE00368A16D9B6A95
:10373000984704227C492000FFF7F4FE61892000AD
:103740000139C9B2FFF77AFE25007849042220002A
:10375000FFF7E8FE00233135EB561421012B00D191
:1037600004392000FFF76AFE260004227049200079
:10377000FFF7D8FE8F2360363370A3686D4A0227A7
:1037800093420BD06C4A934200D0A8E00022AA5684
:10379000CF23012A00D1303B12273370DA212000D9
:1037A000FFF74CFE39002000FFF748FE8121200082
:1037B000FFF744FE31782000FFF740FED9212000BA
:1037C000FFF73CFE0023EB56F121012B00D1CF394E
:1037D0002000FFF733FE200006225849FFF7A2FE23
:1037E000A06A002800D188E00368E16D9B6A9847D1
:1037F000012345E76DB26BE72500270035352878B2
:103800000121363702F01AFF3878012102F016FF45
:10381000002318210126EB56494D4B435A5749487E
:10382000D201121822643200EB185B689A40002320
:103830002265FB564B435A574349D201511812187F
:1038400062643200EB185B68606A9A40130062653C
:103850000A6913430B61002806D0059B002B00D199
:1038600040E70368DB6A3CE72700333731003878EC
:1038700002F0E4FE2300343305931878310002F09F
:10388000DDFE00231821FB562E484B435A57EB18F8
:10389000D2011218A26332005B689A40059BA264B1
:1038A0001B785BB24B435A57ED186B6826499E4014
:1038B000D2015118E6640B691218B343E2630B613D
:1038C00010E7606A002804D00368616EDB69A26EAD
:1038D0009847626C616D13688B43136029E71B4A3C
:1038E0000227934200D059E70022AA56AF23012AAB
:1038F00000D19F3B3370022750E7626C616D136803
:10390000606A0B4313600123002800D1B8E6036806
:103910001B6A98476CE7049B002B00D0E5E604E7A0
:1039200044B6000084B300008CB8000090B80000DA
:1039300094B80000800020008000400098B800008B
:10394000A4B8000010440041004400416000100091
:10395000F0B5140005AA1688002C41DB0A25425F49
:10396000A2423DDD002902DA5B1800211BB20822C9
:10397000855E5A18AA4201DD6B1A1BB2002B2FDD9F
:103980000727E2173A401219D2105543C26A0120A4
:103990003C40A04069185218C0B2012E0CD0002E35
:1039A00013D0022E1CD1013B1BB2591C18D0117828
:1039B000414011700132F6E7013B1BB2591C0FD098
:1039C0001178014311700132F6E7C043C0B2013BE8
:1039D0001BB2591C04D01178014011700132F6E776
:1039E000F0BD0000F0B505AC2588002976DB082481
:1039F000065FB14272DA002A02DA9B1800221BB27B
:103A00000A27C45FD718A74201DDA31A1BB2002BF7
:103A100064DDD2B2DCB2D30873435918C36A5918B3
:103A200007231A401FD001339A1A314BD2B29B5C44
:103A3000944254D2FF26171B3E413340012D06D03D
:103A4000002D08D0022D49D10E78734001E00E7888
:103A500033430B7002E00E789E430E7094423DD3C8
:103A60000826835FC918A31ADBB2072B22D9022DBF
:103A700010D11A000C78083AE4430C700825445F12
:103A8000D2B20919072AF5D80722134026D0194ABD
:103A9000D35C19E02C00621E94411A006442E4B227
:103AA0000C700827C65F083AD2B28919072AF7D8DE
:103AB00007221340002B11D00E4AD35C012D06D0F3
:103AC000002D08D0022D09D10A78534001E00A7870
:103AD00013430B7002E00A789A430A70F0BD012D7F
:103AE000B5D0002DB7D0022DAED08919BBE7C046A6
:103AF0007CB8000084B8000037B5140006AA158809
:103B0000827E022A0DD0032A18D0012A11D1E24365
:103B10000489A41824B20A0000952100FFF762FF6F
:103B20000BE0E2434489C918A418028924B2511A4F
:103B300009B200952200FFF70BFF37BD4289C91873
:103B4000511A09B2E7E737B5140006AA1588827E34
:103B5000022A0DD0032A18D0012A11D10289E418B3
:103B6000141B24B20A0000952100FFF7F1FE0BE0C0
:103B7000CA430189E4188918428909B2141B24B286
:103B800000952200FFF72EFF37BDCA4341898918EF
:103B900009B2E7E7F7B50400806A00284DD0036852
:103BA000A16D9B6A9847052250492000FFF7BAFC97
:103BB000218920000139C9B2FFF740FC07210A23FF
:103BC000E25EA06A0732D3170B409B182289DB10F4
:103BD00053439BB20093E66A002846D0270003684F
:103BE00030373978DB6A9847A06A4021036801259D
:103BF0001B689847009BA06A013B9BB20093009A08
:103C0000036811003A4A914225D0FE2D0CD95B6B16
:103C10009847A06A397803680125DB6A9847A06A4B
:103C2000402103681B689847A06A31780368013512
:103C30001B689847ADB20136DCE7606A002804D003
:103C40000368616EDB69A26E9847626C616D1368F0
:103C50008B431360A7E75B6B9847A06A002838D0B6
:103C60000368E16D9B6A9847F7BD226C216D13686C
:103C700001960B431360009B013B9BB200931A001B
:103C80001B4B9A42E9D0019B606A1978002806D044
:103C900003689B689847019B01330193EBE7082079
:103CA0008025E36BA26BA76C16680D420ED03743DC
:103CB00017601E68E76C01383E431E601E68E76CA3
:103CC0006D08BE431E600028EDD1E4E7BE431660D8
:103CD000EFE7626C616D1368606A0B431360002844
:103CE000C2D003681B6A9847BEE7C0469EB8000072
:103CF000FFFF000010B5024801F09DFE10BDC04658
:103D0000A807002010B5024801F095FE10BDC0467E
:103D100064050020F7B501240326154F1549380026
:103D200000F042F81449154800F03EF814491548CF
:103D300000F03AF81449154800F036F814491548CF
:103D400000F032F8144D1549280000F02DF8390024
:103D50000096230001940022114801F0E5FD009631
:103D6000290001941E231F220E4801F0DDFDF7BD3E
:103D7000EC09002000080042000C0042F409002079
:103D800000100042FC09002000140042040A002038
:103D9000001800420C0A0020140A0020001C0042F7
:103DA000A80700206405002000230371016070470C
:103DB0009446F0B59E1E721E9641624605689207B3
:103DC0002F6836063A4332432A60072505AC24782B
:103DD0000068A4012940214342680024022B00D03E
:103DE0005C03114321434160F0BD30B5C025036839
:103DF000AD031C6812052A402243C0240904A40212
:103E000021401143196003685A6814435C6030BD57
:103E10000123026811680B43136003681A68D20714
:103E2000FCD4DA69D207F9D470470223026811681A
:103E30000B4313600268D3699B07FCD47047026888
:103E4000137E9B0702D40379002BF9D10023037161
:103E50007047002203685A8370470368187E400742
:103E6000C00F70470368187EC0097047802302683E
:103E70005B42117E0B43137670470368588B8007B3
:103E8000C00F704702230268518B0B435383704766
:103E90000368187EC007C00F70470368188DC0B252
:103EA000704703681A7ED207FCD589B219850123B1
:103EB000037118007047012203689A757047012248
:103EC00003681A757047000070B5012604684B0836
:103ED00033403140256809075B070B432B432360C0
:103EE00004685100034802F0F9FC0138C0B22073A5
:103EF00070BDC046006CDC020123026811680B43F0
:103F0000136003681A68D207FCD4DA69D207F9D4BF
:103F100070470223026811680B4313600268D3697B
:103F20009B07FCD470470368DA699207FCD402212E
:103F30001A688A431A607047036818684000C00F07
:103F400070470268936A5B0A5B02194391620368D7
:103F50001A7E5207FCD5986AC0B2704701230268E6
:103F600011680B43136003681A68D207FCD4DA693E
:103F7000D207F9D470470223026811680B4313601B
:103F80000368DA699207FCD430215A8B8A43110006
:103F900010220A435A830268D3695B07FCD4704736
:103FA0000221026813688B4313600268D3699B0780
:103FB000FCD4704780230268DB02116851680B4310
:103FC00053607047036803491A685A680A405A6088
:103FD0007047C046FFFFFBFF032230B50368114066
:103FE0001C68074D5A6809042A40E4061143640F0F
:103FF0005960052C03D10268D3695B07FCD430BD3E
:10400000FFFFFCFF70B5056804006B8B9B069B0FE0
:10401000022B0DD06B8B00209B069B0F032B32D005
:104020006B8B9B0704D56B8B9B069B0F012B2AD1B7
:104030006B6A49001143DB0AC9B2DB020B436B62B6
:104040002368002A13D11A7ED207FCD55B8B9B060E
:104050009B0F022B04D0490800222000FFF7D2FF5B
:104060002368588B4007C30F012058400BE0187E8F
:104070008007C00FF4D11A7ED207F8D5C022596844
:1040800092020A435A6070BD0368283319700268AF
:10409000107EC007C30F508B002B06D1C007C00F86
:1040A00008D1538B9B07F3D570474007C30F0120FE
:1040B0005840F9E71800F7E70368283319700368D8
:1040C00000201A7E520704D5588B01234007C00FE9
:1040D0005840704703681868C006400F04384342D0
:1040E0005841C0B270470368588B8006800F023871
:1040F00043425841C0B270470368187E4007C00F62
:1041000070470368187EC007C00F70470368588B5C
:10411000C006C00F70470368187E8007C00F704745
:104120000368588B0007C00F704703681A68D206EF
:10413000520F052A05D11A7E920702D41A7ED207A1
:10414000F9D528331878C0B2704700000368214AB7
:1041500030B593422FD0204A93422FD01F4A93422A
:104160002FD01F4A93422FD01E4A93422FD01E4A6F
:1041700093421FD10E2319220121032599401B4888
:10418000C024016099082B40AB40FC359D4089005C
:104190000918A4000859A843C0259D402B000343DB
:1041A0000B518023DB011A43114B5A805A7852B2CB
:1041B000002AFBDB30BD09231422DDE70A23152288
:1041C000DAE70B231622D7E70C231722D4E70D23B7
:1041D0001822D1E700080042000C00420010004203
:1041E0000014004200180042001C004200E100E000
:1041F000000C0040F8B504000F0016001D00FFF78A
:10420000A5FF2000FFF704FE1C21BB000B40710737
:104210002268090C0B431360842322689375012FD5
:104220001AD11021012E00D008390C4B69431868AF
:10423000C00002F053FB0722216802408B89520321
:10424000DB04DB0C13438B81226803049089DB0CB5
:10425000400B400318439081F8BDC0463000002059
:10426000F7B50600019308AB1F780D001400FFF7A7
:1042700043FE3000FFF76AFFC0222405920314407A
:10428000BA070C2717433C43C0270722BF022D045F
:1042900033683D4025431D60019B316813401A007F
:1042A00080239B0213434B60F7BD70B504000D00E3
:1042B0001600FFF74BFF2000FFF750FE1C2221687D
:1042C0006D000B6893431A0010231343FF220B6009
:1042D000236815405D62002E04D001232268516AD4
:1042E0000B4353620723226893752268D3695B07E7
:1042F000FCD470BDF8B504000F00FFF727FF2000C5
:10430000FFF72CFE1422236879001A600C4B2568F5
:104310001E68300002F0E2FA0A490400300002F0A0
:10432000DDFA7D23FA215843C90002F0D7FAFF23B2
:10433000241AE868053C1C4098430443EC60F8BD2F
:104340003000002040420F000020704770B50F265B
:10435000CB1D013902003240D5B22C0000093034A7
:10436000092A00DD07341C70013B8B42F2D170BD7D
:1043700010B50C000B4B1868FFF7E8FF21000A4B43
:1043800008311868FFF7E2FF2100084B1031186868
:10439000FFF7DCFF2100064B18311868FFF7D6FF46
:1043A000202010BD0CA0800040A0800044A0800010
:1043B00048A0800008B4024B9C46103808BC6047F7
:1043C00071430000704770473F20704713B56B463C
:1043D0000268D9710733546819000122A04716BD3D
:1043E00070B50A260B7892B06E44023305000B704C
:1043F0003C220021300004F0F1FB394801AC06906A
:10440000384824210790062020776846364AA17450
:104410002281364A364BA281FD3AFF3A8018C17795
:10442000684623390630C17768460730C17702A84D
:10443000C1770720F277032608316944C87703A9BA
:10444000CE7710212B366E443170092621851F311D
:1044500069440E700CA9053E0E703321238002239F
:1044600069440B7006360DA90E7022493536A186B7
:104470003B216E44307010A86274E27702703D32C6
:1044800069446A440B70137040210022E370237169
:104490006371A37341336B44218719705A702B7D6C
:1044A000C039A370A37263770133DBB2A3776A7D4F
:1044B0000B200D0068441543C57731206844037014
:1044C0003A23501C6B441870412302320A436B4458
:1044D0001A7021004222084800F01EFD12B070BD83
:1044E0001001042402060524090400000102000052
:1044F000080B000007050000800A002008B4024BEA
:104500009C46103808BC6047E1430000F8B5027DC6
:104510000B7904000D0000279A420CD10B784E78DD
:10452000A12B0AD1212E06D10100072234311C48CB
:1045300000F0F2FC01373800F8BD212BFBD1202E12
:1045400023D1010007223431154800F01BFC9623CB
:10455000626BDB009A421FD13B342378DB071BD40C
:10456000FA2002F05BF900210D4800F0DDFD012783
:10457000232EE0D1EB78AA781B021343094A0021CD
:104580000748136000F0D0FDD5E7222EEFD10300DD
:104590008A783B331A70DAE702F04AF9E3E7C0465B
:1045A000800A00202800002008B4024B9C461038E6
:1045B00008BC60470D45000010B5343008220021CA
:1045C00004F00CFB10BD000010B5417D006A013104
:1045D00000F002FB034B1B6801335A1E934118186D
:1045E00010BDC0462C00002010B5417D006A02318C
:1045F00000F008FB10BD10B5417D006A023100F0EB
:10460000CFFA10BD70B50D00417D040013000231DA
:104610002A00006A00F0CAFB002801D10123636070
:1046200070BD000010B5054C23685A1C04D1036806
:104630005B69984703002060180010BD2C00002023
:10464000074A0300106810B5411C03D001235B42E8
:10465000136010BD597D186A013100F057FBF8E76F
:104660002C00002070B5050001F0D8FCF423FF33C6
:104670000024984207D93B352C780A20631E9C41C0
:10468000E4B201F001FD200070BD002070477047CA
:1046900070470000FA239B0010B58360114B002285
:1046A000C3820300283383610F4B04004260C26160
:1046B0001800503323610830631D21622060DA77CF
:1046C0000A4A2F3303CA03C38323A362813BE362F5
:1046D0008033236301F0DCFA2100103101F0AAFAE3
:1046E000200010BD03020000FCBC0000F4BC000070
:1046F000022110B5094B1A68437D5B01D318FF33C3
:104700009C7A21439972437D0133DBB25B01D3185C
:104710000122FF33997A0A439A7210BD380F0020A4
:1047200010B502490248FFF7B5FF10BD800A00200E
:104730001C0A0020704710B5040001F02DFD200078
:1047400010BD0000F0B5822919D1C3B2294D5A011C
:10475000AA189169284C80010C40C0218905214389
:1047600091612649083340187021506128685B0127
:104770001A5C8A43110030220A431A54F0BD002902
:10478000FCD1C026C1B21B4C4B01E3189A681A4DEC
:10479000B6052A4032439A60194A800182185A604D
:1047A0000A000727246808325201115DB9430F003F
:1047B0000121394311559F6910493D4040182E434E
:1047C0009E6158617020115D8143080010210143F2
:1047D000115599680B48A2180840802149030143EC
:1047E00099609968890B89039960402311790B437B
:1047F0001371C3E7380F0020FFFFFF8FAC0A0020C2
:104800006C0C0020FF3F00F0EFF3108303600123E6
:10481000436072B670470368002B02D162B6BFF3E3
:104820006F8F704773B5836D0400002B1BD106009A
:10483000A83635786846FFF7E7FF019BEDB2013BEC
:1048400002D33578EDB2FAE768460193FFF7E3FF4C
:10485000002D01D1002076BD2300A4331868A034B8
:104860002368C01AF7E76846FFF7CEFF220000254D
:10487000019BF432013B02D31578EDB2FAE76846AA
:104880000193FFF7C8FF002DE4D02300F033186830
:10489000EC34E5E710B5436D4468DBB25A01A21869
:1048A0009168094808330840802149030143916019
:1048B00091685B01890B890391602268D3184022BB
:1048C00019790A431A7110BDFF3F00F0F7B5436D27
:1048D0004268DBB219000400083110684901411830
:1048E000C979C90711D55B01D21893689B049B0C49
:1048F0000CD12000FFF7CEFF63681A68636DDBB24E
:1049000008335B01D3187F22DA71F7BDE16D00290E
:1049100023D12100A4310B6023000125AC33E565D0
:1049200068465360FFF770FF260020002100019BBE
:10493000A836013BF430F5315A1C33D0357002787B
:104940005F1ED2B20A700A78002A04D120000193B7
:10495000FFF7A0FFE8E73B00EEE72100F0310B6036
:104960000023E3652300603353606846FFF74CFF84
:104970000125260020002100019BF436013BA830D0
:10498000F5315A1C0ED0357002785F1ED2B20A7013
:104990000A78002A04D120000193FFF77BFFE8E7A3
:1049A0003B00EEE768460193FFF735FFA4E737B514
:1049B0006B46DC1D00230D00237001F069F9210016
:1049C00001F0F5F82B681818286020783EBD00002B
:1049D0000078002810D00121084B1B681A898A43EF
:1049E0001A810822198B0A431A830422198B0A435D
:1049F0001A830022024B1A607047C046380F00200D
:104A0000300F002010B50F4A93699B0B9B039361F5
:104A100013680222FF331A729879823A02439A711C
:104A20001A7A9207FCD57F24074A2140937A08001E
:104A3000A3431900802301439172917A5B420B4397
:104A4000937210BD380F00200050004110B50C00CB
:104A500001F01EF9210001F0DDF8002804D1034A1D
:104A600093699B0B9B03936110BDC046380F0020D8
:104A7000F8B50D00832A19D1CBB23B4C5A01A218CC
:104A800091693A48AD010840C0218905014391610F
:104A9000374920686D187021083355615B011A5C35
:104AA0008A43110040220A431A54F8BD022A55D104
:104AB000304A8B009858002802D003685B699847F9
:104AC000F82001F065FB0400274E2B4B4660036085
:104AD00040220021083004F081F822000023A03297
:104AE000A3646565E3642365A365E3655360D364EC
:104AF0001372136013654C3213725372FF222B0032
:104B00001340590171188868184F08330740C020B6
:104B1000800538438860306807265B01195CAD006A
:104B2000B1430E000321314319542300616D6068C5
:104B300011404901411860334B60616D63680A4060
:104B40001B6852019B180122FF33997A20000A4307
:104B50009A72FFF79FFE074B5C51A6E711002800F1
:104B6000FFF7F0FDA1E7C046380F0020FFFFFF8FE1
:104B7000AC0A0020840A002064BD000070B5050066
:104B80000124064BA200D258002A06D0210028009A
:104B90000134FFF76DFF0A2CF3D170BD580A0020D5
:104BA0000B4BCAB20B488901C9185301C31859618C
:104BB00099690832890B89039961036852019A182F
:104BC0000223D3715179823B0B4353717047C04626
:104BD000AC0A0020380F0020084B8A00D05810B5CE
:104BE000002803D003689B68984710BDC9B2044BE6
:104BF0004901591888688004800CF6E7840A00206F
:104C0000380F002010B50C00FFF7E6FF00280CD08D
:104C1000064BE4B21B68083464011C1980236279D6
:104C20005B42134363710223E37110BD380F002010
:104C3000F0B51C00304B85B01B6807000D000292D8
:104C4000002B55D02D4E3178C9B2002902D1192040
:104C500001F040FD64233370294BAA00D05800288E
:104C600008D0036822005B6802999847040020007E
:104C700005B0F0BD29003800FFF7AEFF844204D92B
:104C800029003800FFF7A8FF04000121EBB21D4EF8
:104C900003935B010193F21893689B0B9B03936052
:104CA000019A336802989B18FF335A7A0A435A7262
:104CB000154BA901C918220003F074FF002CD6D0AF
:104CC00029003800FFF788FF0028D0D14021039B3E
:104CD000326808335B01D318187901431971012137
:104CE000D971019BD318FF339A7A0A439A72BEE7AF
:104CF00001246442BBE7C046300F0020A00A002018
:104D0000840A0020380F00206C0C002013B56B467D
:104D1000DC1D22000123FFF78BFF012801D1207841
:104D200016BD01204042FBE770B5CBB2124A1348D2
:104D30005C0189018918021951609168104D08338E
:104D40000D40802149032943402591609168890BDA
:104D50008903916001685A018A18167935431571E3
:104D600095796D06FCD55B01C918CB79DB07FCD5BD
:104D700000198068C0B270BD6C0C0020380F002094
:104D8000FF3F00F070B50D0000211400FFF7CCFFCD
:104D9000A04200D9200000230349A34203D0CA5CEB
:104DA000EA540133F9E770BD6C0C0020F0B51E0029
:104DB0003F4B85B01B680F000192002B3FD0802332
:104DC000DB019E423BD83B4C2178C9B2002902D17D
:104DD0001A2001F07FFC642300252370364BBA01B2
:104DE000D3180293002E2CD0344B1B680393FF235F
:104DF0003B401C0000930834039B64011C19A379F9
:104E0000DB0921D02E4B2F49186801F067FD2E4B8E
:104E10001721584301F062FD2C4BE279920713D41D
:104E2000DA5D002A01D10138F7D20122DA55009B60
:104E30005A01224B9B189A69920B92039A610125A1
:104E40006D42280005B0F0BD0022204B3400DA5539
:104E50003F2E09D9009B40245A01184B9B188022F1
:104E6000996912060A439A6122000199029803F097
:104E700099FE009BA1045A01104B890C9B18029AC1
:104E80002D195A619A69361B920B92030A439A6153
:104E9000009B039A08335B01D3180222DA71597917
:104EA000823A0A435A71019B1B1901939AE7C04643
:104EB000300F0020A10A0020AC0A0020380F00208B
:104EC0003000002040420F0070110100A30A0020B2
:104ED00070B50D001C000D4BAE01F618110030002E
:104EE000220003F05FFEEDB209496D014D196E61BC
:104EF000AB69084A20001340AB61AB69A2049B0B6D
:104F0000920C9B031343AB6170BDC046AC0A0020FA
:104F1000380F0020FF3F00F0F7B5104B01901B78D1
:104F20000F001500002B0CD10D4B16001C78002C27
:104F300009D00C4E0C4834882018641903F032FE56
:104F400034802800FEBD002EFBD03A19330000212A
:104F50000198FFF7BDFF2418361AF4E72C0E002045
:104F60002D0F00202E0F00202D0E0020F8B50F0071
:104F700016000024012A26D9100003F0EDFD0500DB
:104F8000380004F075FB0323022201304000287032
:104F90006B7096420DD9397800290AD0531CDBB2C8
:104FA0000137A9549E4203D00232EC54D2B2F0E74A
:104FB000320029000548FFF7AFFF441EA041C4B2EC
:104FC000280003F0D3FD2000F8BDC046800A002071
:104FD000F0B50024012685B0184B0F0069461E70FD
:104FE00005000094FFF7E3FC154B01A90B806A3B19
:104FF000FF3BCB715A330B72009B8C7109334B8092
:105000000E4B4E7108711C703A00092F0FD00D4FD6
:1050100009223E700C4E280000943480FFF77CFF7C
:1050200069462800FFF7C3FC328808493C70280015
:10503000FFF772FF012005B0F0BDC0462C0E002026
:10504000090200002D0F00202E0F00202D0E002041
:1050500070B5CE7892B005000C00022E0BD18B7982
:10506000C9792C4809021943FFF7B2FF411E884154
:10507000C0B212B070BD00F00BFE210000F0ABFD1D
:10508000002803D0C117081AC00FF2E7012E0ED175
:10509000E279A37912021A431F49112A13D8D2B216
:1050A000002A10D02800FFF737FF0120E1E7032E88
:1050B000DFD1A378002B08D1E279A37912021A4339
:1050C0001649032AEBD90A78ECE7022B08D1E279DA
:1050D000A379120212491A432800FFF747FFC8E7D5
:1050E000012B05D1E279A37912021A430D49F3E7A6
:1050F000032BBED14122010001A803F06FFD00F097
:10510000C7FD01A900F077FDE279A37912021A43E5
:1051100001A9E1E7800A00209EBD00008EBD0000CD
:1051200080BD000092BD0000CBB204495B01C918EC
:105130008B699B0B9B038B617047C046380F002027
:1051400037B5050048780C000B2810D801F0BCFBDF
:10515000061B0F2B0F404561494C5A5D097801AA87
:10516000002906D1022311802800FFF7B1FE01209B
:105170003EBD00231380284B1B78012B00D11370F8
:1051800002230021F0E78A780023012A03D101AA33
:105190001380224BF0E7204A1370214A93699B0B3E
:1051A0009B039361E3E78C78012C06D100211B4B14
:1051B00001AA1C7011702300D6E70120002CD7D162
:1051C000154B174A187093699B0B9B039361CFE7AC
:1051D00089782800FFF716FCC9E72800FFF738FF99
:1051E000C6E701230F4ACCE70B780020DB06BFD1CE
:1051F0002800FFF7C3FCA2780A4B0B481A60FFF7A0
:1052000077FACAE70123094ABBE78A78074B1A6095
:10521000C3E70020ACE7C046A20A0020AA0A00208B
:10522000380F0020300F00201C0A0020340F00200F
:105230004A4BF7B51E780500002E00D07EE0484CA2
:1052400023689A8B12070DD5082231009A8330000B
:10525000FFF778FA10222368FF33997A0A439A728B
:10526000404B1E6023689A8B52071FD504229A83F5
:105270003D4A1378002B0AD01378013BDBB2137040
:105280001378002B03D101211A2001F023FA374AA9
:105290001378002B0AD01378013BDBB2137013781C
:1052A000002B03D10121192001F014FA2368FF33E8
:1052B0001A7A920603D52022597A0A435A721A7A28
:1052C000D20623D569460800294AC0CAC0C0A268D0
:1052D000920B9203A2604022587902435A716023D4
:1052E0000A7828001A422AD1FFF72AFF2368FF33E1
:1052F000002827D08022997952420A439A711A7A5B
:10530000520603D54022597A0A435A727F26012554
:105310002368FF331E722F00236808377F01DB19D3
:10532000DB79002B07D0134BAA00D05800280DD0F2
:1053300003681B6898470135082DECD1F7BDFFF7CE
:1053400085FBD3E720210C4A9171D8E729000B484F
:10535000FFF79EF92368DF19FE71ECE72D0F00209F
:10536000380F0020300F0020A10A0020A00A0020E2
:105370006C0C0020840A0020FF5000411C0A002011
:1053800010B50248FFF754FF10BDC046800A002048
:1053900080235B0003800023436007330372704760
:1053A00083000148C0187047580A0020836C402BC6
:1053B00009D03F22036CC154036C013313400364D2
:1053C000836C013383647047F7B505006846FFF7C7
:1053D0001BFA00264022019B013B02D32E6D961B37
:1053E000FAE768460193FFF716FAAB6D6846002BA3
:1053F0004FD1FFF709FA2900019BA831013B5A1C44
:105400000CD00C785A1EE4B2002C05D168460193EA
:10541000FFF701FA2000FEBD1300F0E76846019394
:105420000024FFF7F8F92A002900A0321368A431FC
:10543000B4420ED0086898420BD92800591CEB18CA
:105440001160603319780830C9B2FFF7AFFF01343B
:10545000E9E709689942DDD1002313600133AB65A8
:105460006846FFF7D1F92F002A000021019BA837D9
:10547000013BF532581CC9D0397010785E1E0028E7
:1054800005D0117028000193FFF704FAEBE7330011
:10549000F0E7FFF7B9F92900019BF431013B5A1CF1
:1054A00006D00C785A1EE4B2002CAFD01300F6E7F9
:1054B000684601930024FFF7AEF92A002900EC3278
:1054C0001368F031B44202D0086898421DD80968C8
:1054D00099429FD1002368461360AB65FFF794F9AA
:1054E0002F002A000021019BF437013BF532581CA4
:1054F00000D18BE7397010785E1E002811D0117032
:1055000028000193FFF7C6F9EAE72800591CEB18B9
:105510001160AC3319780830C9B2FFF747FF013486
:10552000CBE73300E3E710B50400FFF74DFF206D34
:1055300010BD10B50400FFF747FF236D002B03D00B
:10554000E36CE418207A10BD01204042FBE7F7B578
:1055500017000E000400FFF737FF6846FFF754F905
:105560003F2200259446019B013B5A1C19D0BD42A5
:1055700015D2226D002A12D00121226D4942002A43
:105580000AD06046E26CA218117AE26C0132024045
:10559000E264226D013A226571550135E7E7013B6E
:1055A000E3E768460193FFF736F92800FEBD0000E7
:1055B000014B024A1A607047380F0020005000412A
:1055C000F7B50024514B012105001A201C7001F091
:1055D00035F801211A2001F07DF84D4B01211920E9
:1055E0001C7001F02BF80121192001F073F8202321
:1055F000484A0F20D1690B43D361012246490B78F9
:1056000013430B70454B19788143197006211C78A0
:105610002143197042490C7822430A701A780240DB
:105620001A70602219780A431A703E4B3E4A5A801B
:105630005F78FF09FCD13D4800F0EAFC01233C4CB7
:105640003C4E2268300011780B43137080223900E1
:10565000520003F0C3FA22689378DB07FCD4566249
:105660001F26354B1B68590B980C9B01314030406D
:105670005B0FB14200D105211F2800D10238072B52
:1056800000D1043B31408901178D01912B493040F5
:105690000F40019939431185118D0700B14308006E
:1056A00038431085118D1803254B7F260B4003438B
:1056B0000C2013850823D17881430B430321D37039
:1056C0002268D3788B4301390B43D3702268137857
:1056D0003340137004232268167833431370226812
:1056E000C1241389A40083431648138103591B0264
:1056F0001B0A0351802303601378134819430123C5
:1057000011702B700021FEF75DFEF7BDA10A00208D
:10571000A00A002000040040584400413C440041DD
:1057200059440041000C0040064000008153000035
:10573000380F00203C0F0020246080003FF8FFFF5E
:10574000FF8FFFFF00E100E01C0A002001207047EE
:1057500010B50368014A1B6A984710BD1304000086
:10576000FC30006A704787239B00C018C368802004
:105770004000C01A70470300FC331A6A002A03D0A5
:10578000DB69C018007D704701204042FBE710B57F
:1057900004000069FEF73CFB22000023FC32936109
:1057A000D361136287229200A4186360A360E36050
:1057B00010BD872310B59B00C218D368002BFCD105
:1057C0000069FEF73CFB10BDF02001403039484233
:1057D00048417047F0231B011940802306209B009D
:1057E00099420AD00133FF330130994205D080231A
:1057F00002385B00994200D0002070470F20014022
:105800000020012903D00239481E8141481C7047FD
:105810008B23F0B5182685B002919B000400C05C74
:10582000330008214343324D1700EB18595600F05E
:1058300095FF304B0821E05C33004343EB18595689
:1058400000F08CFF2C4BE25C0393022A09D1113348
:10585000E05CFF2805D008214643AE19715600F0E0
:105860007DFF8C26B600A05DFF2819D0012100F035
:10587000E5FE1822A35D21495A43AB56AD18DB0162
:1058800058188D21890060501D4901225B188E2116
:105890008900635069688A408F21890062501A60CC
:1058A0000122029B11002069FEF7A4FC39002000B0
:1058B000FFF790FF390005002000FFF79FFF390038
:1058C00006002000FFF780FF3300009029002069C8
:1058D0000122FEF76DFA0B4B2069E25C039BE15C51
:1058E000FEF783FA2069FEF7A0FA05B0F0BDC046C6
:1058F000A4B800002D0200002F020000184400414F
:10590000144400412E020000802210B50400520011
:10591000002103F063F923000022FC335A602000C9
:105920009A60DA6010BD0000F7B51D0008AB1B7867
:105930000400009309AB1B78160001930023436019
:10594000FA239B008360114B0F000833036014306F
:10595000FFF7DAFF20002130FF30FFF7D5FF8B2360
:105960006A469B002761E654094B1278E554094BBF
:105970002000E2546A46084B1279E2548C22313BF3
:10598000FF3B9200A3541032A354FEBDB0BD0000F3
:105990002D0200002E0200002F020000F7B5EFF3E9
:1059A000108300930123019372B680260200FF2525
:1059B000019BFC327600013B5C1C0FD0D4685F1E5B
:1059C000B44209D054680155546801342C405460E5
:1059D000D4680134D460EEE73B00EDE768460193FC
:1059E000FEF719FFF7BD13B5EFF310830093012302
:1059F000019372B6019B5A1E0192002B15D0030031
:105A0000FC33DA68002A0DD09A68845C9A68013207
:105A1000D2B29A60DA68013ADA606846FEF7FBFEB5
:105A2000200016BD01246442F7E701246846FEF712
:105A3000F2FE6442F4E710B504000069FEF71DFAB7
:105A4000002805D02069FEF728FA2069FEF71AFA27
:105A50002069FEF702FA00281BD02069FEF71DFA24
:105A6000010020001430FFF799FF8C239B00E35CBA
:105A7000FF2B0ED02300FC331A6A80235B009B1A95
:105A8000092B06DC8D238F229B009200E358A2583D
:105A90001A602069FEF7FCF900280ED087239B00CE
:105AA000E318DB68002B14D020002130FF30FFF713
:105AB0009AFFC1B22069FEF7F4F92069FEF7D2F926
:105AC000002805D02069FEF7D1F92069FEF7C1F959
:105AD00010BD2069FEF7F3F9EFE70000F8B5040008
:105AE00000690D00FEF7D4F987239B00E618002813
:105AF00002D0F368002B34D001278022F3685200D3
:105B0000934223D1EFF310833B4210D1174B5B68D4
:105B1000DB05DB0DF1D0103B5BB2002B10DAF13A64
:105B20001340083B9B08124A9B009B181B68206986
:105B3000FEF7AEF90028E0D02000FFF77CFFDCE79D
:105B40009B08C0330B4A9B009B58F0E72000213094
:105B5000FF302900FFF722FF2069FEF7ACF9012092
:105B6000F8BD29002069FEF79CF9F8E700ED00E098
:105B70001CED00E000E100E010B504001430FFF778
:105B800032FF8C239B00E35CFF2B0ED02300FC3301
:105B90001A6A80235B009B1A0A2B06DD8E238F2254
:105BA0009B009200E358A2581A6010BDFEE770B542
:105BB0000E0000254468002C0BD0236831005B6880
:105BC00020009847002802DB2D18E468F3E7012540
:105BD0006D42280070BD70B50D004468002C08D0DF
:105BE000236829009B6820009847002802D1E468B8
:105BF000F4E7200070BD70B50D004468002C07D09C
:105C0000236829002000DB689847E4682D18F5E731
:105C10002C7070BD70B50D004468002C08D023684E
:105C200029001B6820009847002802D1E468F4E7A7
:105C3000200070BDF8B542788B790D00017A9B1871
:105C4000040000208B4222DC6368834219D1656026
:105C5000002623786A71EA792B719B182370AB793F
:105C6000B34213D9AB68B7006078DF19FFF798FB30
:105C70003B68013603606378F6B201336370EEE788
:105C80000B00D9680029FBD1DD60E1E70120F8BDF8
:105C900070B50126054D064C2B68334203D1200018
:105CA000FFF776FB2E60200070BDC0463C10002040
:105CB00040100020F7B506000D000C008B18019372
:105CC000019B671B9C4207D0336821781B6830001A
:105CD000984701340028F3D13800FEBD70B50400A8
:105CE00008000D0003F0C4FC2368020029005B6873
:105CF0002000984770BD10B50B1E02D0FFF7EEFFD5
:105D00000300180010BD10B503688A685B68096855
:105D1000984710BD10B5FFF7EEFF10BD10B5036832
:105D20001B68984710BD000010B50249FFF7D6FF69
:105D300010BDC046E4BD000070B50400FFF7DBFFF6
:105D400005002000FFF7F0FF401970BD70B504009A
:105D5000FFF7D1FF05002000FFF7E6FF401970BDF7
:105D6000F0B58BB06B461500002205330600DA77DC
:105D70000800012D00D80A2509AC290000F034FEE6
:105D8000CAB2130037330700DBB2092902D8130067
:105D90003033DBB2013C2370002FEED12100300004
:105DA000FFF7A9FF0BB0F0BDF8B506000C00151EFB
:105DB00004D10368C9B21B689847F8BD0A2A0CD100
:105DC00000290BDA2D21FFF7A9FF614207002A0005
:105DD0003000FFF7C5FF3818EFE7D2B221003000DE
:105DE000FFF7BEFFE9E710B5FFF7DEFF10BD70B5A6
:105DF0000400FFF7D9FF05002000FFF795FF4019C9
:105E000070BD10B504000068002801D002F0AEFE9D
:105E1000200010BD10B504000068002801D002F079
:105E2000A5FE00232360A360636010BD70B504006D
:105E30000D000068013103F0DFFB031E01D00120DB
:105E400028C470BD036810B50400002B04D043685B
:105E50008B4201D3012010BD2000FFF7E7FF00288F
:105E6000F9D0A368002BF5D122681370F3E770B561
:105E70000E00110004001500FFF7E4FF002804D114
:105E80002000FFF7C7FF200070BD2A003100A56089
:105E9000206802F087FE00232268A1685354F2E7CD
:105EA00070B5050008000C0003F0E2FB21000200C1
:105EB0002800FFF7DCFF70BD10B5002304008AB096
:105EC00023606360A360080001A900F03BF9200093
:105ED00001A9FFF7E5FF20000AB010BD10B50B00C7
:105EE0000400884205D00968002904D09A68FFF7A9
:105EF000BEFF200010BDFFF78DFFFAE7002310B5AD
:105F00000400036043608360FFF7E8FF200010BDDA
:105F1000F7B5040001911600002902D100252800E0
:105F2000FEBD0125002AFAD08368D7183900FFF793
:105F300089FF051EF2D02368A268019998183200E3
:105F400002F030FE00222368A760DA55E7E770B55B
:105F5000050008000C0003F08BFB21000200280064
:105F6000FFF7D6FF70BD002310B5994202D0FFF7AE
:105F7000EEFF0300180010BD10B50400002904D185
:105F80002000FFF747FF200010BDFFF7ECFF0028BF
:105F9000F6D0F8E7FEE70000034B10B51B68002BB6
:105FA00000D0984710BDC0464C10002070B50F4976
:105FB0000F4CA14204D100F0F3F800F0C9F8FEE75D
:105FC0000C4D00238D42F6D0CA18E818A24205D322
:105FD000094B8242EFD00949002204E000680433F3
:105FE0001060F1E704C38B42FCD3E4E7000000201B
:105FF000300200203CC10000300200206C10002064
:1060000010B500F064F8002801D100F055F810BD7B
:10601000014B18607047C0464C100020014B1868B7
:106020007047C04650100020F7B51348012284463F
:106030001249134C8E68636805689B0E13400192E9
:1060400088686268019F920E3A4067463F689342B3
:106050000ED1BD420CD186420AD35B19FA2548689D
:10606000AD00861B07486B437043000DC018FEBD92
:106070003D0013000600E3E75010002010E000E0B0
:1060800000ED00E05555000070B5041E10D0FFF77C
:10609000CBFF050000F01AF8FFF7C6FF054B401BC9
:1060A0009842F7D9FA23013C9B00ED18002CF3D15C
:1060B00070BDC046E703000010B5034A1368013302
:1060C000136000F0BDFB10BD501000207047002091
:1060D0007047F0B50C008BB01600002926D0931E37
:1060E000222B2DD80A2A05D1002803DA01274042A5
:1060F00001AD0AE00027FBE7310000F075FCCBB2F0
:10610000092916D830332B7001352A000028F3D125
:1061100001ABAB42F0D02300002F02D02D21631C35
:10612000217001A98A4206D800221A7020000BB003
:10613000F0BD5733E7E7013A117819700133F0E702
:106140000024F3E710B5FFF7C4FF10BD704700004F
:1061500010B500F0D5F802F0DBFCFFF7F7FF0120E7
:10616000FFF792FF084C2000FFF72AFA2000FEF705
:106170002FFCFCF7BDF8FCF725F8044B002BFAD0F8
:1061800000E000BFF7E7C046800A002000000000E2
:1061900010B502F0E1FC10BD10B502F0E7FC10BD37
:1061A0001E2270B546484749436893431C3A13433F
:1061B000436008238C6923438B61434C434B9C828F
:1061C0009C8A14439C82DC681442FCD00124404A1F
:1061D00014701578254203D055786DB2002DF8DB88
:1061E00001249460547864B2002CFBDB394C546079
:1061F000547864B2002CFBDB8224E4015480547890
:1062000064B2002CFBDB02249C840E34DD68254242
:10621000FCD0314CDC621024DD682542FCD09D8C22
:106220002E4C2C439C841024DD682542FCD0022493
:106230009D8C80262C439C844024DD683542FCD014
:10624000DD682542F9D01024DD682542FCD0002409
:106250009460547864B2002CFBDB214C5460547879
:1062600064B2002CFBDB1C6A1E4D2C4080251C6296
:106270001C6AAC431C62032393601B4B536053782E
:106280005BB2002BFBDB0023FF240B72174A4B721F
:106290008B72CB72164B1A60164B174A1B6811682B
:1062A0009A065B01C90E2340520F12020B4313439F
:1062B000124A1385802342681343436070BDC04671
:1062C00000400041000400400C06000000080040AF
:1062D000000C004001050100B905FF7D040A000023
:1062E00000070300FFFCFFFF03060100006CDC0257
:1062F00030000020246080002060800000400042C8
:10630000FA21314B10B51868890000F0E7FA2F4BDD
:106310000138984256D82E492E4A4860C020136A48
:1063200000061B021B0A03431362002407238C6030
:106330000B608021136A09061B021B0A0B431362C0
:10634000FC22254B196A0A431A62FC22196A92013F
:106350000A431A62A022196AD2020A431A62E0B200
:106360000021013400F06AF9142CF8D11B4B1C00F9
:106370005A7852B2002AFBDB194A5A80194B1A008C
:10638000597EC9090129FBD0E421C90099803F2128
:10639000D970537EDB09012BFBD0C02300205B01A9
:1063A0001361907000F02EF863785BB2002BFBDB7A
:1063B0000D4B0E4A6380D379DB09012BFBD04123BF
:1063C000537010BDFEE7C04630000020FFFFFF0005
:1063D00010E000E000ED00E000040040000C004090
:1063E0001E400000004000422140000000480042E2
:1063F000914202D002D98A1AD0407047521A904076
:10640000FBE70000164A00B51300517EC9090129B7
:10641000FBD00138042816D81969124A0A400F2106
:106420001A615A788A4300F04FFA0308060B0300FA
:10643000110001220A435A7000BD11000322F9E73E
:1064400011000222F6E7F02311691B050B430F210F
:10645000136153788B43190002230B435370EBE70E
:1064600000400042FFFFFFF018234343F0B56A4AA3
:1064700087B09B18DA6806000C000092920722D5BC
:106480001B7C5BB2002B01D0142B1AD1634B0A2268
:1064900019682000FFF7ACFF614A1300D179C909E0
:1064A0000129FBD08005800D1081DA79D209012AFB
:1064B000FBD0022219780A431A70DA79D209012A2C
:1064C000FBD007B0F0BD0827009A544D3A40019226
:1064D00000D191E012229B5E2968200010220193D6
:1064E000FFF786FF019B05001F126B461C79009B7E
:1064F0000421DB0600D40521300000F02FF9494BC0
:10650000BA00D658484BDA5D002A54D10132DA5528
:1065100046490F3202A802F045FB02AA7B009B5AB3
:106520008022D2011A43424B5A805A78D209012A5A
:10653000FBD0022297421BD9338893433380F37BED
:10654000DB09FCD13288403313433380F37BDB0912
:10655000FCD10C34ADB26400A553F37BDB09FCD154
:106560003288023313433380F37BDB09FCD1A8E785
:10657000336893432F4A33601300B1681142FCD152
:106580000222F16B0A43F263B2681A42FCD1103462
:10659000A40034196560B2681A42FCD1264A3264FC
:1065A000B2681A42FCD1022231680A433260B268F2
:1065B0001A42FCD185E7022F07D90C34ADB2640032
:1065C000A553F37BDB09FCD17BE7022372791343EC
:1065D0007371184B1A00B1681942FCD11C34A40025
:1065E000A551B3681342FCD1022331790B433371B7
:1065F000B3681342FCD164E7012100F01FF8296859
:106600003A002000FFF7F4FE01997F2800DD012108
:10661000300000F05FF854E7A4B800003400002018
:10662000004800421000002054100020E8BD000087
:10663000000C0040FF0F7F00FFFF0000182330B563
:106640001D00040045430820204A551928560130F2
:1066500014D0032912D808006343D156D31800F090
:1066600033F902280E1B5868CB010221184A9B18E7
:106670001A1840321170012282405A6030BD5868A9
:10668000CB010621124A9B181A18403211700122C0
:1066900082405A609A61F1E75868CB0106210C4AA2
:1066A0009B181A1840321170012282405A605A61B8
:1066B000E4E75868CB010221054A9B181A184032BA
:1066C0001170012282409A60D8E7C046A4B8000049
:1066D000004400411823F0B508245843114A131808
:1066E0001C5701341BD0012635005F688356BD401E
:1066F0000D4ADB019A18906805420BD10C00601E10
:106700008441D2194032107834400336A400B0439B
:1067100020431070044A9B18002901D15D61F0BD2F
:106720009D61FCE7A4B8000000440041182310B5A7
:106730000824434307490020CA181457013408D0DD
:106740005B560549DB015B18186A5368D840012382
:10675000184010BDA4B80000004400411822424374
:10676000F8B52C4E0300B218127A52B2140001325E
:106770000ED0481C00240C280AD800F0A5F80720E9
:10678000202020202020200B0B0B0B000124644232
:106790002000F8BD092905D10021D8B2FFF74EFF2E
:1067A0000024F5E70A2902D1D8B20839F6E7002417
:1067B0000B29EDD1D8B20A39FFF740FFE8E71820DE
:1067C0004343F2185568F3562C00134ADB016E0858
:1067D00017389B18C9B204409E19002C0DD00F2405
:1067E00030363278090122401143C9B25B19317049
:1067F00040331A7810431870D2E732000F27303236
:1068000016785B19BE433143117040331A78104338
:106810001870BDE7A4B800000044004110B50400A2
:10682000FDF735FF014B1C6010BDC046380000204D
:106830000122024B52421A607047C04638000020C5
:10684000164A10B51368591C26D0013B1360002B63
:1068500022D172B6124B134A0433934213D9124A0F
:1068600001211000147D0C42FCD02021148BFF313B
:106870009B085B0021431183D3610C4B13800123E0
:10688000027D1A42FCD0BFF34F8F094B094ADA60F0
:10689000BFF34F8FC046FDE710BDC0463800002053
:1068A00000200000030200000040004102A5FFFF9D
:1068B00000ED00E00400FA050B0010B5010018001F
:1068C00002F018F910BD000002B4714649084900F1
:1068D000095C49008E4402BC7047C0460022430850
:1068E0008B4274D303098B425FD3030A8B4244D398
:1068F000030B8B4228D3030C8B420DD3FF220902DA
:1069000012BA030C8B4202D31212090265D0030B98
:106910008B4219D300E0090AC30B8B4201D3CB038E
:10692000C01A5241830B8B4201D38B03C01A5241D0
:10693000430B8B4201D34B03C01A5241030B8B42D2
:1069400001D30B03C01A5241C30A8B4201D3CB02BD
:10695000C01A5241830A8B4201D38B02C01A5241A2
:10696000430A8B4201D34B02C01A5241030A8B42A5
:1069700001D30B02C01A5241CDD2C3098B4201D3BD
:10698000CB01C01A524183098B4201D38B01C01A3B
:10699000524143098B4201D34B01C01A52410309B2
:1069A0008B4201D30B01C01A5241C3088B4201D361
:1069B000CB00C01A524183088B4201D38B00C01A0E
:1069C000524143088B4201D34B00C01A5241411A35
:1069D00000D20146524110467047FFE701B5002042
:1069E00000F0F0F802BDC0460029F7D076E7704706
:1069F00003460B437FD4002243088B4274D3030920
:106A00008B425FD3030A8B4244D3030B8B4228D3C0
:106A1000030C8B420DD3FF22090212BA030C8B42E6
:106A200002D31212090265D0030B8B4219D300E086
:106A3000090AC30B8B4201D3CB03C01A5241830B0B
:106A40008B4201D38B03C01A5241430B8B4201D3BB
:106A50004B03C01A5241030B8B4201D30B03C01AE4
:106A60005241C30A8B4201D3CB02C01A5241830A5E
:106A70008B4201D38B02C01A5241430A8B4201D38D
:106A80004B02C01A5241030A8B4201D30B02C01AB7
:106A90005241CDD2C3098B4201D3CB01C01A52411E
:106AA00083098B4201D38B01C01A524143098B42A7
:106AB00001D34B01C01A524103098B4201D30B0190
:106AC000C01A5241C3088B4201D3CB00C01A5241B5
:106AD00083088B4201D38B00C01A524143088B427A
:106AE00001D34B00C01A5241411A00D20146524113
:106AF000104670475DE0CA0F00D04942031000D332
:106B00004042534000229C4603098B422DD3030A86
:106B10008B4212D3FC22890112BA030A8B420CD396
:106B2000890192118B4208D3890192118B4204D3BF
:106B300089013AD0921100E08909C3098B4201D33F
:106B4000CB01C01A524183098B4201D38B01C01A79
:106B5000524143098B4201D34B01C01A52410309F0
:106B60008B4201D30B01C01A5241C3088B4201D39F
:106B7000CB00C01A524183088B4201D38B00C01A4C
:106B80005241D9D243088B4201D34B00C01A524123
:106B9000411A00D20146634652415B10104601D3B0
:106BA0004042002B00D54942704763465B1000D33A
:106BB000404201B5002000F005F802BD0029F8D0E0
:106BC00016E770477047C0468446101C62468C46E4
:106BD000191C634600E0C0461FB500F0F1FF002815
:106BE00001D40021C8421FBD10B500F049FF40424A
:106BF000013010BD10B500F0E3FF002801DB0020DC
:106C000010BD012010BDC04610B500F0D9FF00280E
:106C100001DD002010BD012010BDC04610B500F000
:106C20006BFF002801DC002010BD012010BDC04614
:106C300010B500F061FF002801DA002010BD01202E
:106C400010BDC0468446081C6146FFE71FB500F032
:106C5000A9F8002801D40021C8421FBD10B500F0DA
:106C60002BF84042013010BD10B500F09BF8002811
:106C700001DB002010BD012010BDC04610B500F0A2
:106C800091F8002801DD002010BD012010BDC04694
:106C900010B500F039F8002801DC002010BD0120FB
:106CA00010BDC04610B500F02FF8002801DA002012
:106CB00010BD012010BDC04670B542004E024C0010
:106CC00045026D0A120EC30F760A240EC90FFF2A61
:106CD0000FD0FF2C11D00120A24200D070BDB542D0
:106CE000FCD18B420DD0002AF8D12800451EA841C6
:106CF000F4E70120002DF1D1EBE70120002EEDD1CA
:106D0000E9E70020EAE7C04670B54A004E024502B6
:106D100044006D0A240EC30F760A120EC90FFF2C11
:106D200015D0FF2A0ED0002C15D1002A01D1002E3B
:106D30001CD0002D14D08B4227D00220013B1840DC
:106D4000013870BD002EEED002204042F9E7002D40
:106D5000FAD1FF2A0ED0002A0ED1002EEDD00BE082
:106D600001230139994308000130EAE70020002D92
:106D7000E7D0E2E7002EE7D18B42DED1944205DD79
:106D80000221581E08400138DBE70024A24204DC3F
:106D9000B542D2D80020B542D3D2581E0123984321
:106DA0000130CEE730B5420044024D02C30F480027
:106DB000640A120E6D0A000EC90FFF2A12D0FF28B6
:106DC0000CD0002A12D1002819D1002D17D1002C87
:106DD0002BD00220013B1840013826E0002DF0D0D6
:106DE000022022E0002CFBD1FF281FD000281FD159
:106DF000002D1DD10220013B1840013815E0002C68
:106E00000ED08B42E5D10022904204DCAC42E0D8A7
:106E10000020AC4209D2581E01239843013004E0FF
:106E20000123013999430800013030BD002DD7D12D
:106E30008B42CED18242E7DD0221581E0840013844
:106E4000F3E7C046F0B54F464646D6460C00090368
:106E5000C0B5490A470F5E0039431F03DB0F9C464C
:106E600065007B0A570F1F436D0DE40F760DA14699
:106E7000C000B846D200AB1B64457BD0002B5FDD61
:106E8000002E00D0A4E03E00164300D112E15E1EA9
:106E9000002E00D09EE1871A4346B842804101256A
:106EA000C91A4042091A0B0200D431E149024E0AC4
:106EB000002E00D16EE1300001F0FEFD0300083B22
:106EC0001F2B00DD61E120223900D21A9E40D14003
:106ED0009F400E439D4200DD51E15D1B6B1C1F2B4B
:106EE00000DD7CE12021C91A3D0030008F40884040
:106EF000DD40791E8F41310007222843D94000250B
:106F000007433A40002A09D00F233B40042B05D009
:106F10003B1DBB42BF417F42C9191F000B0200D479
:106F200026E26A1CC64B55056D0D9A4200D106E15A
:106F3000C44AFF080A40530752023B43120B8EE03B
:106F4000002B00D0B8E06B1C5B055B0D012B00DC57
:106F500030E1871A4346B842B641CB1A76429E1BAF
:106F6000330200D54CE13B003343A1D10022002481
:106F7000002570E0002B00DCE5E0002E00D183E06E
:106F8000AF4EB54260D0802636043743B846382B22
:106F900000DC3EE1434613431F007A1E97413F1831
:106FA00087428041404209180B0200D4B0E0A44B54
:106FB00001359D4200D1C3E0A24A7B080A4001216D
:106FC0000F401F435108D30707221F433A4099E758
:106FD0009B4EB54238D0802636043743B846382B0E
:106FE00000DDDCE01F2B00DC30E11E004746203EC8
:106FF000F740BC46202B04D04026F31A46469E405C
:107000003243170063467A1E97411F43CCE0002BA2
:1070100000D104E24346134300D159E14B07C008B5
:1070200018438023C9081B03194208D04546ED08C0
:107030001D4204D14346D008590708432900420F96
:10704000C9007F4D1143C0004B07CA087C49C008E6
:1070500003438D4268D012036D05120B6D0D0021A4
:1070600012031800130B0A0D12051A43764B2D0557
:1070700013402B435B00E4075B08234319001CBC4F
:1070800090469946A246F0BD3E00164312D05E1EC1
:10709000002E00D000E187188742804141444042E1
:1070A000091801250B0233D5022585E76446330014
:1070B000414610001D00C7E7002D00D0DAE00C00AB
:1070C0000443F3D05C1C00D19FE15D4CA64200D18B
:1070D0002FE1DB43382B00DD66E11F2B00DD83E170
:1070E00020240500E41A0F00DD40D940A0404346AB
:1070F000A7405B1A441EA04198462F433843171AF5
:10710000BA42924143465242991A64463500CAE651
:1071100007223A40002A00D0F6E64B07CA08484941
:10712000FF083B438D4296D11900114300D19EE1E7
:10713000802109030A431203120B414D8FE715000A
:10714000002200238BE7002B00D0C7E06B1C5F05FB
:107150007F0D012F00DCF1E0394DAB4200D1B9E0E9
:1071600085180A0085428941424449425118072244
:10717000CF076D082F4349083A401D00C2E6072299
:107180003049ED1A31403A40BCE63E00283886408E
:1071900000279FE6380001F08FFC20308EE6434642
:1071A00013431F007A1E9741C71BB84280414042DB
:1071B000091A78E60E003B0006431343002D61D107
:1071C000002E00D0F4E0002B00D11BE16446390012
:1071D000100039E71A4FBB427AD03300FFE6300087
:1071E0001F3DE840202B03D04021CB1A9E4037435F
:1071F0007B1E9F41072207433A400021002589E773
:10720000171A4346BA42B641591A76428E1B644653
:107210004EE61F2B00DDADE020264746F61AB740AC
:10722000B9461700B246DF404E463E433700564649
:10723000B240561EB24117434246DA408918AEE6C4
:10724000FF070000FFFF7FFFFFFF0F80202647465C
:10725000F61AB740B9461700B246DF404E463E43E5
:1072600037005646B240561EB24117434246DA40F6
:10727000891A99E77F4CA6425BD0802424045B42A4
:10728000214327E7002E0CD1002B00D1CBE0644630
:1072900039001000774DD7E6764FBB4218D0330047
:1072A00075E6002B14D04B07C00818438023C9088B
:1072B0001B03194207D0FC081C4204D17907D008EF
:1072C0000843E14621004C46420FC9001143C0006B
:1072D000684DB9E61D0000220023C0E6002D5BD1F9
:1072E0000D00054300D1E2E65D1C00D1B0E0614D28
:1072F000AE421FD0DB43382B71DC1F2B00DD96E044
:1073000020250F00ED1AAF40B9460700AA46DF401E
:107310004D463D432F005546A840D940451EA84143
:1073200088440743BF189742924151424144350077
:107330003AE6644635004146100085E60B000343FB
:10734000002D00D063E6002BF5D04346134300D157
:107350007AE6871887428041072241444042091853
:107360003A400B0200D4D5E6434B01351940C9E53C
:10737000380069E61E004746203EF740BC46202BF9
:1073800004D04026F31A46469E4032431700634617
:107390007A1E97411F4302E6364DAE42CAD0802581
:1073A0002D045B422943A6E70843411E8841A6E617
:1073B000002B00D148E6871A4346B842B641CB1AA3
:1073C00076429E1B33024BD5171A4346BA4292416E
:1073D000591A5242891A072264463A4092E50143FB
:1073E0000F00791E8F419DE71C000F00203CE740F5
:1073F000202B03D04024E31A99400843411E8841C2
:1074000038437CE60022002425E6171A4346BA4298
:107410009241591A5242891A6446350043E5414661
:107420001000144D10E680220024120380E61D0097
:107430000F00203DEF40BC46202B03D04025EB1A27
:107440009940084307006346781E87411F4369E758
:10745000871897429B4141445B42C9183500A3E518
:107460003B003343CED0072231003A4052E600239E
:107470001A00F4E5FF070000FFFF7FFFF0B5574655
:10748000DE464E464546E0B5834607000E034800FB
:1074900085B092461C00360B400DCD0F002800D160
:1074A0009DE0954B984239D08023F6001B041E4383
:1074B000924A7B0F334399469446030063440093FA
:1074C00000230026FF00029323031B0B9846630052
:1074D000E40F52465B0D019400D1B3E086498B4224
:1074E00000D19EE04246D100802212040A43514658
:1074F000490F11438B46814952468C46009963449B
:10750000CB1A0021D20000932B0063409A460F2E25
:1075100000D905E17A4BB6009B599F465B46334341
:10752000994600D0B8E00223082600270090029375
:10753000CAE7CB463A0002990195019B9A46022977
:1075400027D0032900D180E2012944D06D49009B56
:107550008C4663441C00002C38DD530700D013E236
:10756000D2085B46DB0109D55946674B19408B466B
:107570008021C9008C46009B63441C00634B9C42E5
:1075800007DC5B4664055F075B0217431B0B620D5C
:1075900002E000230027584A00211B031C0B0B0D9F
:1075A0001B05234314055A4A380013401C43534615
:1075B0006400DB0764081C43210005B03CBC904616
:1075C0009946A246AB46F0BD0122524201231B1B45
:1075D000382B00DCADE1002200230027DCE75B460E
:1075E000334399465ED0002E00D18AE1300001F08D
:1075F00063FA03000B3B1C2B00DD7BE11D22D31A39
:107600005A460100DA4008398E4013005F46334382
:1076100099468F403F4B00261B1A0093002302938C
:1076200052E7414653460B433B499B468C46009BE1
:10763000634400935B46002B3BD1022300221E4390
:10764000022161E7434613439B4637D04346002B54
:1076500000D162E1404601F02FFA03000B3B1C2BE6
:1076600000DD53E102004146083A914088461D2161
:10767000CB1A5146D9400B0041460B439B4653461B
:1076800093401A00009B25499C46604403008C46A9
:1076900063440093002137E70323B14600900C2692
:1076A000029311E70023009301330426002702937D
:1076B0000AE70323C3461E43032125E701331E4384
:1076C0000022012120E700239A46802300271B0384
:1076D000094A61E7802349461B03194200D1E2E0D1
:1076E0005946194200D0DEE00B431B0317001B0B69
:1076F000A246014A50E7C046FF07000001FCFFFF19
:10770000F8BD0000FF030000FFFFFFFEFE070000C2
:10771000FFFF0F800DFCFFFF01F8FFFFF3030000E8
:10772000D94500D9CBE000D1C6E03C00484600274F
:10773000009B013B00935B46160E1B021E43130287
:10774000984633041B0C9946310C0191FFF74CF914
:107750004A4642430B04210C050019438A4207D9CB
:107760008919013D8E4203D88A4201D9851E8919A3
:10777000881A0199FFF738F909048C464A46210412
:1077800064464243090C030021438A4204D9891903
:10779000013B8E4200D8F1E02D041D43AB46434629
:1077A000891A4246280C12041D0C5B46140C220058
:1077B0001B041B0C5A4303946B43444302956843D8
:1077C0001B19150CEB189C4203D980246402A446B3
:1077D00060441C0C15041B042D0C20185D198142FB
:1077E00077D373D00C1AA24A7D1BAF42BF41944697
:1077F000009B7F426344E01B1C00864200D1DBE01B
:107800000199FFF7F1F84A4642430B04290C07009F
:1078100019438A4207D98919013F8E4203D88A4207
:1078200001D9871E8919881A0199FFF7DDF8090423
:107830004A46894629044D464243090C0300294320
:107840008A4207D98919013B8E4203D88A4201D95D
:10785000831E89193F04891A3A00039F1A4338008E
:1078600013041B0C584381460298150C6F43434385
:1078700045434846000C8446DB1963449F4203D9C4
:10788000802040028446654448461F0C00041B04C7
:10789000000C7D191818A94200D284E000D17FE0C5
:1078A00001231A4357E680234A461B0313431B0355
:1078B0001B0BAA466F4A6FE6BA4200D935E74B4622
:1078C000DC0758087B081C43FF0734E70024AF425D
:1078D00089D247444745A4415B466442A4196418D1
:1078E000013BA6421ED2A0426DD800D1B6E0241AB8
:1078F0009B4678E703005A46283B9A40002791466A
:1079000088E6584601F0D8F8203072E60300524667
:10791000283B9A4093460022B4E6504601F0CCF84A
:1079200020309AE6A642E2D1B845DCD9341A9B460B
:1079300059E71F2B65DC504C0099A4465C46614416
:1079400008008C4011008240D940501E82410C43F7
:1079500014435A46DA401300620709D00F2222402E
:10796000042A05D02200141D9442894149425B1823
:107970001A0262D50122002300270DE68A4200D8B0
:107980000AE7831E891907E70F231340042B00D150
:10799000E6E5171D9742924153429B44FA08E0E501
:1079A000002800D1D7E57118531EB14227D3A94250
:1079B00015D358D01A0073E7002B00DC04E601232E
:1079C00000229B44CDE502234744474589415B4261
:1079D0009C46494289190C19E344241A03E743469B
:1079E0005F0047459B41B8465B429E19023A8919A0
:1079F000A94200D054E7404500D051E7ABE51A005A
:107A0000F6E71F215F4649420C1BE740202B07D0B9
:107A10001A49009B8C46634418005B4683401A4316
:107A2000501E82413A4307270023174009D00F21F7
:107A3000002311401400042995D122005F075B0246
:107A40001B0BD20817430022A6E5802359461B03CF
:107A50000B431B0317001B0B064A9DE5BD42B2D822
:107A60009B460024BFE68045B9D31A00C3E7C04651
:107A7000FF030000FF0700001E0400003E0400009A
:107A8000F0B54F464646D6468446C0B58046194EA8
:107A900018030F034D00000B5C0082463F0B6D0D79
:107AA000C90F9146640DDB0F0120B5420AD0B442E4
:107AB00003D0A54201D157450CD01CBC9046994635
:107AC000A246F0BD66463E43F7D1AC42F5D15446DE
:107AD0001443F2D10120C845EFD1994207D0002DBF
:107AE000EBD163461F433800471EB841E5E700204D
:107AF000E3E7C046FF070000F0B54F464646D646CE
:107B00004D00C0B50E03C90F8A462C491F035C0007
:107B10008046360B6D0D91463F0B640DDB0F8D4299
:107B20001ED08C4216D0002D1ED130438446002C2E
:107B300001D13A4323D06246002A1AD09A4529D06F
:107B4000514602200139084001381CBC9046994634
:107B5000A246F0BD39001143E5D002204042F4E7CF
:107B60003043FAD1AC420FD0002C0FD13A43E7D0CA
:107B70000CE00122013B934318000130E5E7634626
:107B80000020002BE1D0DBE73A43E6D19A45D7D17C
:107B9000A542D5DCA54205DBBE42D1D808D00020E5
:107BA000BE42D2D250460123013898430130CCE77F
:107BB000C845C5D80020C845F4D3C6E7FF07000074
:107BC000F0B54F464646D6464D00C0B50E03C90F28
:107BD0008A462E491F035C008046360B6D0D914688
:107BE0003F0B640DDB0F8D4218D08C4211D0002D5D
:107BF00018D130438446002C1ED13A431CD1634631
:107C00000020002B30D051460220013908400138B5
:107C10002AE039001143EAD0022025E03043FBD1AD
:107C2000AC4226D0002C26D13A4324D15146022022
:107C300001390840013817E06246002A0FD09A4502
:107C4000E1D1A54205DBBE42DDD819D00020BE42FD
:107C50000AD25046012301389843013004E0012242
:107C6000013B9343180001301CBC90469946A24644
:107C7000F0BD3A43D0D19A45C5D1A542C3DCE0E777
:107C8000C845C0D80020C845E3D3EDE7FF07000092
:107C9000F0B55746DE464E464546E0B583460600FB
:107CA0000F03480087B092461D003F0B400DCC0FDC
:107CB000002800D16FE0DE4B984238D08023FF00CF
:107CC0001B041F43730F3B430193DA4B0027994674
:107CD00000239B46F60081442B0369001B0B524690
:107CE0009846490DED0F002900D185E0D04B99420F
:107CF00000D173E04346DA0080231B04134352464D
:107D0000CC48520F84461343524600206144D200AF
:107D100089442100694000918C46012149448A46EA
:107D20000F2F00D990E0C449BF00CF59BF465B4632
:107D30003B43019300D06AE10223082700268146D5
:107D40009B46C9E732005846019B614600910228D4
:107D500000D175E0032800D1FEE1012800D02CE11C
:107D600000230027002600253F032A0D3F0BB348C0
:107D700012053A4302401B051343009A5B00D107EA
:107D80005B080B433000190007B03CBC9046994695
:107D9000A246AB46F0BD5B463B43019300D12FE1C9
:107DA000002F00D1A5E1380000F086FE03000B3B58
:107DB0001C2B00DD96E11D22D31A5A460100DA4041
:107DC0005E4608398F4013008E403B4301939C4B25
:107DD00000271B1A994600239B467DE741465346E0
:107DE0000B4393498C46E144002B00D01AE1022258
:107DF0000220174300228CE7134300D10DE14346D4
:107E0000002B00D181E1404600F056FE02000B3A03
:107E10001C2A00DD72E10100434608398B40984678
:107E20001D239A1A5346D3401A0043461343524621
:107E30008A404946081A824989468144002068E7F9
:107E40007B4B002700268EE7140C1204120C110045
:107E5000370C3604350C794328008C462E006043DD
:107E60006044834656432100300C8046584679438F
:107E700040440291844506D98846802149028C46B7
:107E8000E044414602913604010C360C00048B4656
:107E900081191E0C1B041B0C0391190079438C469D
:107EA000280075436544A8465843050C454477436C
:107EB000A94203D9802149028C466744290C8C468B
:107EC00039000004000C2D042D186144AB440591C9
:107ED0005946049101990F043F0C080C3900514395
:107EE0004243904602008C46090C8B4662437C4319
:107EF00044445C44A04503D9802149028846424459
:107F0000210C884661460904090C8C463900594306
:107F1000434370437E430F0CF6182404BE19644497
:107F200042448C46B34203D980235B0298464044C6
:107F3000029B61469846049B370443449B46AB45ED
:107F4000AD416B420D0405992D0C8C467F19674499
:107F5000FD18A8465D462D19A542A44193466442EA
:107F6000A446C344DC448F42BF4198459B4193459E
:107F70009241A445A4415B427F421F43360C5242CA
:107F80006442BF192243BF18624638184302D20D1B
:107F9000039913436A020A43501E82416146ED0D64
:107FA0002A434E023243D90100D4B3E001265008DF
:107FB00032400243DE0732435B08224C5444002C1B
:107FC00062DD510709D00F201040042805D0101D94
:107FD0009042924152429B180200D90104D580245C
:107FE0001948E400034054441848844200DD27E760
:107FF0005E075B02D2081F0B630516435B0DB2E6FA
:10800000002399460133042700269B4664E6032398
:10801000019781460C279B465EE60122012017430B
:10802000002276E6032303201F43434671E6C04641
:10803000FF07000001FCFFFF38BE0000FFFF0F80BC
:108040000DFCFFFFFF030000FFFFFFFEFE07000027
:108050000023802700933F030026434B83E6019BC8
:108060003200A446584670E6AC466EE68027019979
:108070003F0339422DD03B422BD11F433F033F0BDF
:1080800000951600384B6EE601252D1B382D00DDBE
:1080900066E61F2D40DC35481C0050441600824027
:1080A0008440EE40501E824134431443EB4062074B
:1080B00009D00F222240042A05D02200141D944228
:1080C000804140421B181A023ED50123002700269A
:1080D00049E68027019B3F031F433F033F0B00946A
:1080E000214B40E603005A46283B9A400026019265
:1080F0006DE6584600F0E0FC203057E6030052469B
:10810000283B9A401300002293E6504600F0D4FC2E
:1081100020307BE6CA4650E71F201E004042041B69
:10812000E640202D03D0124C5444A3401A43501E65
:108130008241324307260027164009D00F20002332
:10814000104014000428B9D122005E075B021F0B07
:10815000D2081643002306E680273F031F433F0350
:108160003F0B1600004BFEE5FF0700001E04000059
:108170003E040000F8B557464E464546DE460C0024
:108180000903E0B5490A460F5F0031431E03DB0FC8
:10819000760A9B46530F3343C84E6500C000E40F78
:1081A000D2006D0DA24681467F0D9C469046B74297
:1081B00000D1B9E05B46012673409B46EE1BA34508
:1081C00000D183E0002E63DD002F00D0B1E06346D4
:1081D000134300D123E1731E002B00D0BAE1861AAD
:1081E0006346B04280410125C91A4042091A0B0278
:1081F00000D447E149024B0A98464346002B00D180
:1082000089E1404600F058FC0300083B1F2B00DDCD
:108210007CE120223000D21A4146D0409940020031
:108220009E400A439D4200DD6AE15D1B6B1C1F2BD3
:1082300000DD94E1202110003500C91A8E40DA409B
:108240008840DD40711E8E41110007222843002521
:1082500006433240002A09D00F233340042B05D0B7
:10826000331DB342B641764289191E000B0200D479
:108270003DE26A1C914B55056D0D9A4200D119E102
:108280008F4AF6080A40570752023743120B9BE009
:10829000002E00D0C5E06E1C7605760D012E00DCA8
:1082A00048E16746861ACB1BB042BF417F42B846C1
:1082B0001F004346FF1A3B00B8461B0200D55FE192
:1082C00037439AD100220024002579E0002E00DCFB
:1082D000FAE0002F00D18DE0784B9D4267D08023DB
:1082E00067461B041F43BC46382E00DC52E1634640
:1082F00013435A1E93411E1886428041404209187A
:108300000B0200D4BEE06D4B01359D4200D1D2E09E
:108310006B4A73080A4001210E401E435108D307DF
:1083200007221E43324095E71E00164300D045E762
:1083300040E7624B9D423AD0802367461B041F43AF
:10834000BC46382E00DDEBE01F2E00DC3AE13300A6
:108350006746203BDF403B00202E05D04027BF1B57
:108360006646BE40324390464646721E96413343AF
:10837000DAE0002B00D114E26346134300D168E138
:1083800080234E07C008C9081B030643194208D0C2
:108390006046C008184204D163460100D2085E0757
:1083A0001643F3009946C900720F444D11434B46E2
:1083B000DE08424B4F073743CA089D4200D16EE0AA
:1083C00012036D05120B6D0D00211203130B0A0D24
:1083D00012051A433B4B2D0513402B435B00E4076A
:1083E0005B082343380019003CBC90469946A246DE
:1083F000AB46F8BD6346134311D0731E002B00D06B
:1084000007E18618864280416144404209180125EF
:108410000B0237D502257BE73E00614691463500C9
:10842000C5E75C46002D00D0E1E00B000343F3D02C
:10843000731C00D1ACE1214B9F4200D13AE1F343E0
:10844000382B00DD6FE11F2B00DD8CE120250E00B5
:10845000ED1AAE40B0460600AA46DE40454635431A
:108460002E005546D940A8406346451EA8415B1AD8
:108470009C463043161AB242924163465242991AC0
:108480003D00B4E607223240002A00D0E4E60B4B60
:10849000F6084F073743CA089D4200D090E73B00DB
:1084A000134300D1A6E180231B031A431203120BCE
:1084B000024D89E715000022002785E7FF0700002D
:1084C000FFFF7FFFFFFF0F80002E00D0C7E06B1C77
:1084D0005E05760D012E00DCF0E0C84DAB4200D108
:1084E000B9E085180A008542894162444942511821
:1084F0000722CE076D082E43490832401D00A9E629
:10850000BF49ED1A114007223240A3E63200283855
:108510008240002686E6300000F0CEFA203073E676
:10852000634613435A1E9341C61AB04280414042EB
:10853000091A5CE60E00674606431743002D5ED11C
:10854000002E00D0F3E0002F00D11EE15C46614612
:1085500091462CE7A94FBE427BD01E00F1E61000E9
:108560001F3DE840202B03D04021CB1A9A401643F0
:10857000731E9E410722064332400021002583E7F7
:10858000161A6346B2428041591A40420B1A984665
:108590005C4632E61F2E00DDABE02027BB1B9A466F
:1085A00063465746BB40994613004F46F3401F436E
:1085B0003B005746BA40571EBA4113436246F24049
:1085C000891898E62027BB1B9A4663465746BB404E
:1085D000994613004F46F3401F433B005746BA40AD
:1085E000571EBA4113436246F240891A9CE7834BF7
:1085F0009F425FD080252D047342294320E7002E3F
:108600000CD1002F00D1D0E05C46614691467B4DF5
:10861000CDE67A4FBE421CD01E0065E6002F18D072
:10862000C0084E0706438020C9080003014208D055
:108630006346DC08044204D12100DA46D2085E0712
:108640001643F300994601245346C900720F1143A3
:108650001C406A4DABE61D0000220027B4E6002D49
:1086600059D10B00034300D1D6E6731C00D1B2E010
:10867000624B9F421ED0F343382B6FDC1F2B00DD73
:1086800097E020250E00ED1AAE40B0460600AA463F
:10869000DE40454635432E005546A840D940451E8C
:1086A000A8418C440643B618964292415142614417
:1086B0003D0025E63D006146914678E60B00034308
:1086C000002D00D055E6002BF5D06346134300D1B2
:1086D0006DE68618864280416144404209180022B6
:1086E0000B0200D4D0E6464B01351940B2E5B14645
:1086F0005DE633006746203BDF403B00202E05D07F
:108700004027BF1B6646BE40324390464646721E17
:1087100096413343EFE5394B9F42CBD080252D0462
:1087200073422943A8E70843411E8841A2E6002F6F
:1087300000D13CE66346861ACF1AB0429B415B42A9
:10874000FB1A98461B024ED5161A6346B242924156
:10875000591A5242891A5C4600227BE501430E00F9
:10876000711E8E419FE71D000E00203DEE40B04679
:10877000202B04D04025EB1A9940084381464846F7
:108780004346411E8841184374E60022002417E640
:10879000161A6346B2429241591A5242891A3D0052
:1087A00025E561469146154D01E68022002412031D
:1087B00079E61D000E00203DEE40B046202B04D08F
:1087C0004025EB1A9940084381464E464346711EA8
:1087D0008E411E4367E7861896429B4161445B4287
:1087E000C9183D008CE547463743CED007224146A5
:1087F000324049E600273A00E6E5C046FF070000A0
:10880000FFFF7FFF70B50C4E0D031C0349005B009A
:108810002D0B490D240B5B0DB14208D006490020F9
:108820008B4203D114432000441EA04170BD054378
:108830000120002DFAD1F1E7FF07000030B5144DFB
:108840000A034B00120B5B0DC90F0024AB4211DD74
:10885000104CA34210DC8024640322430E4CE41A23
:108860001F2C0CDD0D48C31ADA4013005C420029AE
:1088700000D11C00200030BD094BCC18FAE7094D8F
:10888000E040AC4663449A4013000343EEE7C04621
:10889000FE0300001D040000330400001304000068
:1088A000FFFFFF7FEDFBFFFF10B5041E25D000F09A
:1088B00003F9144B1B1A5B055B0D0A2812DD0B38FC
:1088C000844000222403240B0021100024030A0DFD
:1088D000240B120522430C4C1B05224013435B0062
:1088E000590810BD02002100153291400A000B21E9
:1088F000081AC4402403240BE6E7002300240022C6
:10890000E2E7C0461E040000FFFF0F804100090E91
:108910004B1C70B5DBB24602750AC40F012B14DD87
:10892000E0239B006D07360BCB1800210A0D2800B1
:1089300012051C4D32435B052A405B0813435B0064
:10894000E4075B082343190070BD002914D1002DF2
:108950001ED0280000F0B0F80A281CDC0B232A00E7
:108960001B1ADA40030015339D400F4B12031B1AEC
:108970005B05160B5B0DD8E7002D06D0320B802669
:1089800036036D071643094BCFE7084B0026CCE7AB
:1089900000230026C9E703002A000B3B9A4000256C
:1089A000E3E7C046FFFF0F8089030000FF070000D8
:1089B000F0B54C00640D0B03621C5B0A460F5205B8
:1089C000C90F1E43C500520D012A29DD374BE71898
:1089D000FE2F1CDC002F3BDD8001431E9841072247
:1089E000F3006D0F03432B431A40002A04D00F22DB
:1089F0001A40042A00D004338022D2041A4024D022
:108A00000137FAB2FF2F02D09B01580A01E0FF2282
:108A100000204002D205400AC90710430843F0BDB8
:108A20003543002C04D1002D0AD100220020F0E7AC
:108A3000002DECD08020C0033043FF22E9E7002462
:108A400000235B02580AE2B2E3E7DB083C00F8E7E8
:108A50003B001733F3DB80231B0433431E26F61B36
:108A60001F2E14DD02225242D71B1A00FA401700B3
:108A7000202E04D00E4A94466444A3401D432B008C
:108A80005D1EAB4107223B431A400027ADE7094A70
:108A90002800A218954093406C1EA541F040072283
:108AA0002B4303431A4000279FE7C04680FCFFFF8B
:108AB000A2FCFFFF82FCFFFF1C2101231B04984244
:108AC00001D3000C10391B0A984201D3000A08395F
:108AD0001B09984201D30009043902A2105C401816
:108AE0007047C046040302020101010100000000BA
:108AF0000000000010B5040004481300002804D052
:108B00000A000220210000E000BF10BD00000000AC
:108B100070B500260C4D0D4C641BA410A64209D163
:108B2000002602F003F90A4D0A4C641BA410A64269
:108B300005D170BDB300EB5898470136EEE7B3009E
:108B4000EB5898470136F2E70C0200200C02002097
:108B50000C0200202802002010B5034B0100186809
:108B600000F08EF810BDC0463C00002010B5034B4D
:108B70000100186800F03AF810BDC0463C00002023
:108B800082B0002900D101A9101E06D0002B06D00A
:108B900013780B601078431E984102B07047022092
:108BA0004042FAE7002310B59A4200D110BDCC5CD8
:108BB000C4540133F8E710B5884202D98B189842A3
:108BC00003D3002307E08B5C8354013AFBD210BD32
:108BD000CC5CC45401339A42FAD1F8E7030012186E
:108BE000934200D1704719700133F9E770B5050061
:108BF000002910D00C1F2368002B00DAE41828008D
:108C000001F0C7FB1D4A1368002B05D16360146097
:108C1000280001F0BFFB70BDA34209D9216860188C
:108C20008342F3D118685B6841182160EEE71300B6
:108C30005A68002A01D0A242F9D919685818A042EE
:108C40000BD120680918581819608242E0D11068C9
:108C50005268411819605A60DAE7A04202D90C2321
:108C60002B60D5E721686018824203D110685268F2
:108C70004118216062605C60CAE7C0465C10002059
:108C8000032370B5CD1C9D43083506000C2D1ED264
:108C90000C25A9421DD8300001F07BFB254A146841
:108CA0002100002919D1244C2368002B03D1300066
:108CB00000F0ACFC20602900300000F0A7FC431C51
:108CC0002BD10C233000336001F064FB03E0002D56
:108CD000DFDA0C233360002070BD0B685B1B19D4F6
:108CE0000B2B03D90B60CC18256003E04B688C423A
:108CF0000DD11360300001F04DFB200007220B3036
:108D0000231D9043C31AE7D05A42E250E4E7636060
:108D10000C00EFE70C004968C3E70323C41C9C4325
:108D2000A042E1D0211A300000F070FC431CDBD1DE
:108D3000C7E7C0465C10002060100020F0B58BB083
:108D400014001D1E129953DA802424061B191D00DD
:108D500014002D230B702023149E03229E43462EC5
:108D600007D03300453B59424B411099013ACB188B
:108D7000109309AB049308AB0393139B00920293E7
:108D8000109B220001932B0000F00CFD0700472EE2
:108D900002D1119BDB0724D5109BFB180793462EAD
:108DA00014D13B78302B0CD1002200232000290065
:108DB000FDF71AFF002804D10123109A9B1A139A79
:108DC0001360139B079A1B68D31807930022002394
:108DD00020002900FDF708FF302200280DD0079B56
:108DE00009933800099B159ADB1B13600BB0F0BD8B
:108DF0000023AFE7591C09911A70099B07998B4210
:108E0000F8D3EEE7F0B5831C85B0019306000C00A3
:108E100002702B23002901DA2D234C427370092C98
:108E200022DD02ABDD1D20000A21FDF7C7FE6F1E0B
:108E30003031397020000A21FDF7DAFD04000928DD
:108E40000BDC023D3034019B2C7002AA0732180063
:108E5000AA4204D8801B05B0F0BD3D00E3E72A78A4
:108E600001351A700133F0E73023E418B370301D78
:108E7000F470EFE7F0B595B00C000A920B931A9DD1
:108E8000099001F06FFA036818000C9300F0F0FBF2
:108E90000023129323680E900D930D99277E2B6863
:108EA0000722C90545D59B1893431A0008322A604A
:108EB0001A685B68A264E3640122E56CA66C6B002F
:108EC0005B080F935242AC4B30000F99FFF79AFCAE
:108ED000002830D10122A84B524230000F99FDF7F3
:108EE00093FE002827D10022002330002900FDF73F
:108EF00081FE002803D023002D2243331A709F4D9A
:108F0000472F00D89E4D032300260D9A236101337D
:108F10009A4322600B9B13AA009321000A9B099895
:108F200000F0F4F9431C00D093E00120404215B05A
:108F3000F0BD0733B8E732002B0030002900FFF7FF
:108F400061FC002804D08F4D472FDCD88E4DDAE726
:108F500080230D996268DB000B43511C43D107321B
:108F6000626012AA0021059211AA039223222360B3
:108F70000691019308A96368521802920093320087
:108F80002B0004970998FFF7D9FE20233A0005002B
:108F90009A43472A07D1119BDA1C02DB626893428D
:108FA00045DD023FFFB21199652F25D82000013918
:108FB0003A0050301191FFF725FF129A060013185E
:108FC0002361012A02DC2268D20701D50133236123
:108FD000232308AA9B181B78002B9BD023002D224B
:108FE00043331A7096E7672F00D176E1472FB8D147
:108FF000002AB6D10122B3E7662F19D16368002990
:109000000CDD2161002B02D12268D20702D5013389
:109010005B182361119B0026A365D9E7002B03D1C0
:1090200001222168114200D09A1C2261F2E76727D1
:10903000119B129A934205DB22682361D207E9D57E
:109040000133E6E70121002B01DC4918C91A521847
:10905000EBE72268530508D423692A000A99099886
:109060000B9DA847431C29D15FE7652F00D8E0E09E
:10907000A06CE16C00220023FDF7B6FD002834D07F
:109080000123424A0A9909980B9DA847431C00D125
:109090004BE7119B129A934202DB2368DB070DD545
:1090A0000B9D0E9B0C9A0A990998A8470025431C12
:1090B00000D13AE7129B013BAB420ADC23689B07D5
:1090C00000D508E1139BE068984200DB2FE7180009
:1090D0002DE7220001231A320A9909980B9EB04706
:1090E000431C00D121E70135E4E7119B002B2DDC67
:1090F0000123264A0A9909980B9EB047431C00D1C8
:1091000013E7119B002B05D1129B002B02D1236882
:10911000DB07D3D50B9E0E9B0C9A0A990998B04792
:109120000026431C00D100E7119B5B42B34201DCE7
:10913000129B92E7220001231A320A9909980B9F89
:10914000B847431C00D1F0E60136EDE7A36D129F4E
:109150009F4200DD1F00002F08DD3B002A000A9916
:1091600009980B9EB047431C00D1DEE600230D9307
:10917000FB43DB170F9318E0FFFFEF7F86BE000075
:1091800082BE00008EBE00008ABE000092BE0000BB
:10919000220001231A320A9909980B9EB047431CFA
:1091A00000D1C2E60D9B01330D930F9BA66D0D9A66
:1091B0003B40F31A9342EBDC119B129AAD19934298
:1091C00010DB2368DB070DD4129F119BBE1BFF1A17
:1091D000B74200DD3700002F0DDCFE43F3170025FA
:1091E0000C931CE00E9B0C9A0A9909980B9FB847A8
:1091F000431CE9D199E63B002A000A9909980B9D86
:10920000A847431CE9D190E6220001231A320A99AB
:1092100009980B9EB047431C00D186E60135119A90
:10922000129B0C999B1A3A000A409B1AAB42EBDC4A
:1092300044E7129B012B02DC01231A4232D00123A6
:109240002A000A9909980B9FB847431C00D16CE685
:109250000E9B0C9A0A9909980B9F0135B847431C3D
:1092600000D162E6A06CE16C129B00225F1E00231D
:10927000FDF7BAFC3B00002814D000250AE02200CC
:1092800001231A320A9909980B9FB847431C00D151
:109290004BE60135129B013BAB42F0DC2200330070
:1092A0005032DBE62A000A9909980B9DA847431C17
:1092B000F4D13AE62200012319320A9909980B9E4B
:1092C000B047431C00D130E60135E368139A9B1A7E
:1092D000AB42EFDCF6E60025F7E7002A00D189E68D
:1092E0000021069112A9059111A90391232108A833
:1092F00009182360019300922B0004970291320019
:109300000998FFF71BFD050045E6C046F7B51500B7
:1093100001938A680B6900900C00934200DA1300F5
:1093200022002B6043321278002A01D001332B60D7
:1093300023689B0602D52B6802332B60062723681F
:109340001F4027D0230043331B785A1E93412268C5
:10935000920630D42200019943320098089EB0470B
:10936000431C25D0062320682A68E16803400025B5
:10937000042B03D18D1AEB43DB171D40A368226930
:10938000934201DD9B1AED180027BD4220D1002039
:1093900010E00137E3682A689B1ABB42D2DD220045
:1093A0000123193201990098089EB047431CF0D15F
:1093B00001204042FEBD3020E118433108702100F9
:1093C0005A1C45310978A218433202331170C1E7A3
:1093D000220001231A3201990098089EB047431CCD
:1093E000E6D00137D1E70000F0B589B004920A0059
:1093F00043320593039002920A7E0C000E9B6E2A64
:1094000000D186E01FD8632A33D008D8002A00D1C3
:109410008CE0582A4DD0250042352A7030E0642A6D
:1094200001D0692AF7D1196825680A1D280629D5AF
:1094300008681A60002803DA2D23029A404213704C
:109440006B4E0A274FE0732A74D008D86F2A1FD0BA
:10945000702AE0D1202209680A43226003E0752ABD
:1094600016D0782AD7D12200782145321170614E6A
:1094700022E025001A684235111D196013682B700F
:10948000012365E008681A606906D3D500B2D1E708
:1094900019682568081D186008682E0605D5544E01
:1094A00008276F2A1BD00A2719E06D06F7D580B26E
:1094B000F5E745314E4E0A7018682268011D0068B4
:1094C0001960150621D5D30702D520231A4322603F
:1094D0001027002803D1202322689A43226023000A
:1094E000002243331A706368A360002B58DB042208
:1094F000216891432160002854D1029D002B5AD04D
:109500002500337842352B7055E05506DBD580B207
:10951000D9E71A680D68101D4969186013682E068E
:1095200001D5196002E06D06FBD519800023029D6C
:1095300023614FE01A68111D1960156800216268E7
:10954000280000F01BFF002801D0401B606063680A
:1095500023610023029A13703CE023692A000499D6
:109560000398059DA847431C3ED023689B0715D44C
:10957000079BE068984239DA180037E0220001239F
:10958000193204990398059EB047431C2CD001352D
:10959000E368079A9B1AAB42F0DCE9E70025F7E79E
:1095A0000028ADD0029D3900FDF71EFA735C013D25
:1095B0002B700028F7D1082F09D12368DB0706D5C7
:1095C00063682269934202DC3023013D2B70029BC9
:1095D0005B1B2361059B07AA00932100049B039852
:1095E000FFF794FE431CB8D10120404209B0F0BD02
:1095F00094BE0000A5BE000010B5034B0A00010098
:10960000186801F0BDF910BD3C000020002370B5C2
:10961000064C05000800236001F07AFB431C03D1CF
:109620002368002B00D02B6070BDC046681000205E
:109630000EB400B50B499CB01DAB0290069007918B
:1096400004910948094904CB0591006802A90193D6
:1096500001F01EFA0023029A13701CB008BC03B07C
:109660001847C046FFFFFF7F3C0000200802FFFFB5
:109670000023C25C0133002AFBD1581E70470B1E29
:1096800004D0FF2A04D98A2303608B3B180070475B
:109690000A700123FAE7F0B503690C6989B0070085
:1096A00005910026A34265DB0B00013C1433A500A5
:1096B00003935B1904930300143302935D19049B15
:1096C00028681B68591C0193FDF708F90190B04206
:1096D00029D0039B02989C460696624608CA944687
:1096E000019A99B251431B0C534389190A0C9B18D8
:1096F00007931E0C036889B29AB2069BD2180368BE
:10970000521A190C6B469B8BCB1A11145B18191447
:1097100092B21B041A43049B069104C06345DCD239
:109720002B68002B2DD00599380001F049F800284E
:109730001FDB0025019B0298013303990193026806
:1097400008C992B255199AB2AA1A05681B0C2D0CB9
:10975000EB1A15145B191D1492B21B04134308C0B5
:10976000049B8B42EBD2029AA300D3181A68002AFA
:1097700011D0019E300009B0F0BD2B68002B04D140
:10978000013C029B043DAB42F7D33C61CBE71A6836
:10979000002A04D1013C029A043B9A42F7D33C616F
:1097A000E7E70000F0B516001F00446A9BB0029086
:1097B000239D06960797002C08D11020FFF7CCF9BF
:1097C000029B5862446084600460C460029B5B6AD0
:1097D000196800290BD05A68012393404A608B60B6
:1097E000029800F010FE0022029B5B6A1A60002FB4
:1097F00020DA01232B607B005B080793079CB24BA8
:10980000220017931A409A4217D1B04B229A136044
:10981000069B002B03D1240301D100F087FDAC4B44
:10982000249A0893002A02D0AA4B249A136008981D
:109830001BB0F0BD00232B60E0E7069E079F0022CF
:10984000002330003900FDF7CFF9051E0BD00123AE
:10985000229A1360A04B249A0893002AE7D09F4ACB
:1098600024990A60E3E718AB019319AB0093320027
:109870003B00029801F022F8630003905B0D74D066
:109880003A03974C120B14432100964A3000169568
:109890009E180022944BFEF76DFC944A944BFEF701
:1098A000F7F9944A944BFDF7CDFA040030000D000F
:1098B00001F0F4F9914A924BFEF7EAF902000B002D
:1098C00020002900FDF7BEFA04000D00FEF7B6FFE8
:1098D00000220700002320002900FDF78BF9002853
:1098E00009D0380001F0DAF92B002200FDF77CF9ED
:1098F000434258413F1A01231493162F0DD8814932
:10990000FB00C91808684968069A079BFDF786F9A5
:10991000002846D00023013F1493189B9E1B002370
:109920000A933300013B0B9304D501239B1B0A933D
:1099300000230B93002F36DB0B9B1197DB190B9346
:1099400000230493209B0124092B00D984E0052BDC
:1099500002DD0024043B2093209B981E032800D99D
:1099600084E0FCF7B1FF7577286A189B199A9E1856
:10997000654BF218202A0FDD40239B1A9C40634B55
:109980000698F318D8402043FEF78EFF0123604C61
:10999000013E091916937CE7202306989B1A9840EC
:1099A000F2E71490B9E70A9BDB1B0A937B4204930E
:1099B00000231193C6E701230D93219B002B59DD52
:1099C0000C930993029A556A00226A6004321000CF
:1099D00014306968984252D9029800F0DCFC029B6E
:1099E00028605B6A1B680893099B0E2B00D90AE16B
:1099F000002C00D107E1069B079C12931394002FC3
:109A000000DC89E00F213A003E4B0A40D2009B184F
:109A10001D685E6802233C110E93E3060BD53D4B97
:109A20000C401A6A5B6A12981399FDF727FD03230D
:109A3000069007910E9300233AE001230D93219B9A
:109A4000FB180C9301330993002BBBDC0123B9E70E
:109A50000023B1E70023F1E700230D942093013B9D
:109A600000220C93099313332192ABE701230D934A
:109A7000023BF5E701230C9309931A00F4E7013147
:109A800069605200A3E701231C420ED00E9B214ABD
:109A900001330E93109B2800DB009B1831001A68DD
:109AA0005B68FEF7F5F805000E00109B64100133AB
:109AB0001093002CE7D1069807992A003300FDF790
:109AC000DDFC0690079142E00000F07F0F270000C8
:109AD000C0BF0000C3BF000092BE000093BE0000E4
:109AE0000000F03F01FCFFFF0000F83F61436F639F
:109AF000A787D23FB3C8608B288AC63FFB799F50A7
:109B00001344D33F50C00000320400001204000090
:109B1000000010FE28C0000002230E93002F16D074
:109B2000129813997C420D332340CE4ADB00D318A0
:109B30001A685B68FEF7ACF8002301261D0006904A
:109B400007912411002C00D08CE0002BB9D1149B7C
:109B5000002B00D196E0069C079D0022C24B2000FE
:109B60002900FDF747F8002800D18BE0099B002B66
:109B700000D187E00C9B002B41DDBC4B0022200074
:109B80002900FEF785F80E9B0690079101330E938E
:109B90000C9B7E1E0E98109301F080F8069A079B8E
:109BA000FEF776F80022B24BFDF74CF9B14A0E9061
:109BB0000F910E9C0F9D94460F9B634415931D00BF
:109BC000109B002B61D1069807990022AA4BFEF743
:109BD000D1FA2200159B06900791FDF71FF8002887
:109BE00000D0A8E2A5480F99844661440B0006986E
:109BF00007992200FCF7FEFF002800D095E2129B97
:109C0000139C06930794199B002B00DA5CE10E2F3E
:109C100000DD59E1934BFA009B185C681B680493C4
:109C20000594219B002B00DBD8E0099B002B00DD75
:109C3000D4E000D07DE20498059900228E4BFEF717
:109C400027F8069A079BFCF7F3FF099B04931E0075
:109C5000002800D04FE2089B089A5D1C3123013791
:109C600013704BE234420AD00E9B854A01330E93A7
:109C7000EB009B181A685B68FEF70AF83300641063
:109C800001355FE73E00099B84E7109B0D995A1E42
:109C9000744BD2009B181A685B68002949D00020D9
:109CA0007849FDF7EBFB2B002200FEF763FA089BD7
:109CB0000E900F91159306980799FEF7BFFD0400CB
:109CC00000F0ECFF02000B0006980799FEF752FA2D
:109CD000159B30345D1C1C700E9A0F9B06900791EB
:109CE000FCF788FF00286CD1069A079B00205E498C
:109CF000FEF740FA0E9A0F9BFCF77CFF002800D07D
:109D0000C3E0089B109AEB1A9A4200DC77E70E98A2
:109D10000F990022554BFDF7BBFF00220E900F91CB
:109D200006980799514BFDF7B3FF159506900791DB
:109D3000C1E720002900FDF7ABFF089C109A230023
:109D400094460E900F916344159306980799FEF779
:109D500075FD050000F0A2FF0B00020006980799B0
:109D6000FEF708FA3035159B2570013406900791EF
:109D7000A3422AD10E980F99089A109B94466344E7
:109D800000221D003F4BFDF75DF802000B00069816
:109D90000799FCF743FF002800D076E00E9A0F9B4E
:109DA00000203849FEF7E6F902000B0006980799F3
:109DB000FCF720FF002800D121E76B1E1A78302A1B
:109DC00001D037003FE01D00F7E706980799002211
:109DD000264BFDF75DFF06900791B6E7089E049AB3
:109DE000059B06980799FDF749FBFEF727FD040040
:109DF00000F054FF049A059BFDF74AFF02000B0098
:109E000006980799FEF7B6F9230030333370099AA4
:109E1000089B751CEB1A9A4248D102000B00FDF713
:109E200011F8049A059B06900791FCF7F7FE0028AD
:109E30002AD1049A059B06980799FCF7D5FE0028BD
:109E400001D0E30720D40399029800F0DCFA002344
:109E50002B70229B01371F60249B002B00D1E6E46E
:109E60001D60E4E450C000000000F03F000024400A
:109E700000001C400000C0FC000014400000C07C3A
:109E800028C000000000E03F3E006B1E1A78392A0F
:109E900006D1089A9A4207D1302313701300013675
:109EA0001A7801321A708CE71D00EEE70022A44BED
:109EB000FDF7EEFE00220023069007912E00FCF72E
:109EC00093FE00288BD0BEE70D9A002A00D1DAE07D
:109ED000209A012A00DDBDE0169A002A00D1B5E0E3
:109EE000984A9B18049D0A9C0A9A0121D2180A924A
:109EF0000B9A0298D3180B9300F025FB0600002C58
:109F00000EDD0B9B002B0BDD0B9A2300944200DD32
:109F100013000A9AE41AD21A0A920B9AD31A0B93D4
:109F2000049B002B1FD00D9B002B00D1AFE0002D18
:109F300011D031002A00029800F09EFB039A010024
:109F40000600029800F008FB03991090029800F0B8
:109F50005AFA109B0393049B5A1B04D0039902984E
:109F600000F08AFB03900121029800F0ECFA119BAB
:109F70000490002B00D1E3E11A000100029800F0E8
:109F80007BFB209B0490012B00DD82E00025069BDB
:109F9000AB420ED1079B1B03AB420AD1179B079A1A
:109FA000134206D00A9B013501330A930B9B013300
:109FB0000B93119B0120002B6CD10B9B18181F23B6
:109FC00018407ED001331B1A042B70DD1C23181A95
:109FD0000A9B24181B180A930B9B1B180B930A9BB4
:109FE000002B05DD1A000399029800F097FB0390FF
:109FF0000B9B002B05DD1A000499029800F08EFBE4
:10A000000490149B002B5ED00499039800F0D8FBB9
:10A01000002858DA00230A220399029800F00CFA6B
:10A020000D9B013F0390002B00D190E100233100F4
:10A030000A22029800F000FA0C9B0600002B00DDBB
:10A0400088E0209B022B00DC84E044E03623189A51
:10A050009B1A47E7099B5D1E049BAB4208DB5D1B17
:10A06000099B002B0CDA0A9B099A9C1A00233BE7F8
:10A07000049B0495EA1A119B00259B181193EFE7A6
:10A080000A9C099B30E7049D0A9C0D9E37E7049AC1
:10A0900064E70025049B049A1B69109303339B001B
:10A0A000D318586800F006FA2023181A85E7042B05
:10A0B00095D00A9A1C33D2180A920B9AE418D31836
:10A0C0008CE70300F5E7099B002B3DDC209B022B6E
:10A0D0003ADD099B0C930C9B002B0CD104990522B3
:10A0E000029800F0A9F904900100039800F068FBC1
:10A0F000002800DDAFE5219B089DDF430023099385
:10A100000499029800F07FF9002E00D19BE6099B8C
:10A11000002B05D0B34203D01900029800F073F968
:10A120003100029800F06FF98DE6109B04931E0039
:10A13000E1E70023FAE7109B370004931E008AE54D
:10A1400000002440330400000D9B002B00D1B2E03E
:10A15000099B0C93002C05DD31002200029800F0D1
:10A16000DDFA06003000002D11D07168029800F071
:10A1700012F93100040033690C319A1C92000C3042
:10A18000FEF710FD01222100029800F0C7FA09969F
:10A190000600089B0A9304990398FFF77CFA099933
:10A1A0000D900400039800F00BFB3200109004990E
:10A1B000029800F01FFB01230B93C36830340500A5
:10A1C000002B04D10100039800F0FAFA0B9029004B
:10A1D000029800F018F90B9B209A13430ED1069AAF
:10A1E000013313420AD1392C26D0109B002B01DDFC
:10A1F0000D9C31340A9B5D1C1C7081E7109B002B69
:10A2000007DB1D00209B1D4322D10123069A134228
:10A210001ED10B9B002BEDDD03990122029800F06B
:10A220007DFA0499039000F0CBFA002802DCE1D11A
:10A23000E307DFD5392CDBD10A9B0A9A5D1C392351
:10A2400013706B1E1A78392A67D001321A7057E7DB
:10A250000A9B5D1C0B9B002B04DD392CECD00134D8
:10A260000A9BC9E70A9B0C9A1C70089BEB1A934245
:10A270003ED000230A220399029800F0DDF8099BE2
:10A280000390B34209D100230A220999029800F0F1
:10A29000D3F8099006000A957DE7099900230A2260
:10A2A000029800F0C9F8002309900A2231000298B0
:10A2B00000F0C2F8EEE7099B0C93089B0693049903
:10A2C0000398FFF7E8F9069B30305D1C18700C9A74
:10A2D000089B0400EB1A9A4208DD00230A22039926
:10A2E000029800F0A9F806950390E8E70023099387
:10A2F00003990122029800F011FA0499039000F0EA
:10A300005FFA00289DDC01D1E3079AD46B1E1A780E
:10A31000302A00D0F4E61D00F8E7089A9A4203D1EB
:10A32000312301371370EBE61D008AE70B4B249AAB
:10A3300008930B4B002A01D0FFF777FAFFF777FA63
:10A34000209B012B00DC21E6119D012035E60C9BB2
:10A35000002BB2DC209B022BAFDDBCE6B7BF0000B8
:10A36000BFBF0000034B1B68186A002800D10248D9
:10A37000F03070473C000020A0000020C9B28218D5
:10A38000904201D10020704703788B42FBD001300E
:10A39000F6E77047704770B5466A04000D00002E5E
:10A3A00007D11020FEF7D8FB606246608660066029
:10A3B000C660666AF368002B13D0636AAA00DB6884
:10A3C0009B181868002818D101210E00AE40721D9C
:10A3D0009200200000F0C6FA00280CD0456086608C
:10A3E0000DE021220421200000F0BCFA636AF06035
:10A3F000DB68002BE1D1002070BD02681A600023E9
:10A400000361C360F8E770B5446A06000D00002CD4
:10A4100007D11020FEF7A0FB7062446084600460E6
:10A42000C460002D07D0736A6A68DB6892009B18CD
:10A430001A682A601D6070BDF7B51E0014239C4683
:10A4400007000C0000200D698C4463461B68013036
:10A4500099B263461B6851431B0C534389190E0C78
:10A460009B1989B21E0C1B045B18614608C18C46FF
:10A470008542EADC002E1BD0A368AB4212DC636885
:10A480003800591CFFF787FF2100236901909A1CAF
:10A4900092000C310C30FEF785FB21003800FFF7ED
:10A4A000B2FF019C2B1D9B00E31801355E60256106
:10A4B0002000FEBD0300020C0020824201D11B04DB
:10A4C00010301A0E01D108301B021A0F01D10430CE
:10A4D0001B019A0F01D102309B00002B03DB0130DE
:10A4E0005B0000D4202070470722036810B50100EC
:10A4F0001A400DD001240020234205D1023003422E
:10A5000003D0E34020000B6010BD9B080B60FBE70D
:10A510009CB21000002C01D110201B0CDAB2002AD2
:10A5200001D108301B0A1A0701D104301B099A0710
:10A5300001D102309B08DA07E8D45B0801D0013072
:10A54000E4E72020E0E710B50C000121FFF723FF2E
:10A5500001234461036110BDF0B50B691400126959
:10A5600089B00D00934201DA25000C002F6926699D
:10A570006968BB190293AB68BA19934200DA0131DA
:10A58000FFF709FF0200BB1914329B00D3189C4649
:10A5900000211300049063451DD31435BF00EB194F
:10A5A0001434B6000593A319039501940793079BF0
:10A5B0000199994211D3029B002B06DD04235B42D3
:10A5C0009C4463461B68002B51D0049B029A1800E0
:10A5D0001A6109B0F0BD02C3DDE7019B1B6898B2A8
:10A5E00000281CD015000026039F02CF2C688BB2D8
:10A5F0004343090C4143A4B21B199B190E0029685F
:10A600000695090C71181E0C89190E0C9BB20904D1
:10A610000B4308C5059BBB42E7D8069B5E60019BC8
:10A620001B681D0C1ED0100000271368039E3168A4
:10A63000046889B26943240C0919C9190F049BB233
:10A640003B43036080CE43683F0C6F439BB2FB18D3
:10A65000090C5B18059906901F0C0430B142E6D82E
:10A6600006994B60019B0432043301939FE7029BE0
:10A67000013B02939FE700000323F7B51340050059
:10A680000E001400002B08D02249013B9A005258BA
:10A6900000233100FFF7D0FE0600A310019336D04F
:10A6A0006C6A002C07D11020FEF756FA68624460ED
:10A6B00084600460C4606F6ABC68002C07D11649CE
:10A6C0002800FFF740FF00230400B8600360012268
:10A6D000019B13420AD0310022002800FFF73CFF03
:10A6E000070031002800FFF78EFE3E00019B5B1043
:10A6F00001930CD02068002807D1220021002800F7
:10A70000FFF72AFF0023206003600400DFE730002A
:10A71000FEBDC04618C1000071020000F0B50D007A
:10A7200017002B69541185B0E3180193013300938E
:10A730004968AB680290009A934235DB0298FFF7B4
:10A740002AFE00230200060019001432A3422EDB69
:10A75000E343DB171C402B00A40014192A691433AF
:10A7600092009A1894461F22174024D00132D21B1F
:10A770000392002219682000B9400A4304C404CBA4
:10A780000399CA409C45F5D84260002A02D0019B3B
:10A7900002330093009B0298013B33612900FFF7CD
:10A7A00032FE300005B0F0BD01315B00C3E7980018
:10A7B00011500133CAE704CB04C49C45FBD8E9E738
:10A7C0000A69036930B59B1A0DD192001430143117
:10A7D00084188918043C043925680A68954204D015
:10A7E0000123954204D3180030BDA042F2D3FAE70A
:10A7F0005B42F8E7F0B50D0085B0070011002800B6
:10A800001400FFF7DDFF061E08D101003800FFF736
:10A81000C2FD01234661036105B0F0BD0123019330
:10A82000002804DB23002C001D0000230193616835
:10A830003800FFF7B0FD2F000022019B2669C3609E
:10A840001434B300E31802932B6914379B00FB18F0
:10A85000039303009446143320CC04CF0192AAB290
:10A8600094446A46614692882D0C8A1A0199090C13
:10A87000691A151449190D1492B209040A431A6091
:10A88000039AAC460433BA42E6D802991A008C42C5
:10A8900005D3043A1368002B0ED00661BCE704CC44
:10A8A00091B261440D14120C5219151489B212049C
:10A8B0000A43AC4604C3E8E7013EEAE7F7B51D00EA
:10A8C00001211400089FFFF766FD2B036D000600B1
:10A8D0001B0B6D0D24D10193002C27D068460094EA
:10A8E000FFF702FE009C00281ED0019B20211A00C9
:10A8F000091A8A40C340224372610193019CB461EA
:10A90000631E9C4101343461002D18D0124BED18A8
:10A9100035232D183D60181A099B18603000FEBDC4
:10A92000802252031343D6E77461E7E701A8FFF7DB
:10A93000DBFD0124019B346173612030E4E7074BA8
:10A94000C018074B3860E3189B00F3185869FFF7ED
:10A95000B1FD6401201ADFE7CDFBFFFFCEFBFFFF57
:10A96000FFFFFF3F4A4370B511001400FEF788F95E
:10A97000051E03D022000021FEF730F9280070BD2B
:10A98000F8B507000D001600002905D11100FEF7EB
:10A9900077F904002000F8BD002A03D1FEF726F95C
:10A9A0003400F7E700F072F92C00B042F2D2310027
:10A9B0003800FEF765F9041EECD029003200FEF7DE
:10A9C000F1F829003800FEF711F9E3E7F0B58E68D9
:10A9D00085B007000C00039201939E423CD890235F
:10A9E0008A89DB001A4234D00325096923685B1A7F
:10A9F0000293636902985D43EB0F5D19019B6D1033
:10AA000001331B18AB4200D91D00530532D5290074
:10AA10003800FEF735F9061E09D10C233B604023B0
:10AA20000120A28940421343A38105B0F0BD029AE0
:10AA30002169FEF7B7F8A389144A1A40802313430B
:10AA4000A381029B2661F61826606561019EED1ABE
:10AA5000A560019B9E4200D9019E320003992068A7
:10AA6000FEF7A9F8A36800209B1BA36023689E192A
:10AA70002660DAE72A003800FFF782FF061EE0D1E1
:10AA800021693800FEF7B2F8C7E7C0467FFBFFFF39
:10AA9000F0B59FB0029005938B890F0016001B063E
:10AAA00011D50B69002B0ED14021FEF7E9F8386073
:10AAB0003861002805D10C23029A013813601FB0B9
:10AAC000F0BD40237B61002306AC636120336376D5
:10AAD0001033A37635002B78002B01D0252B46D1DF
:10AAE000AB1B04930CD0320039000298FFF76EFFC5
:10AAF000431C00D1AEE06269049B944663446361E9
:10AB00002B78002B00D1A5E0012200235242626085
:10AB100002A9543252186E1C2360E360A3601370C4
:10AB2000A365317805225448FFF728FC751C0028DE
:10AB30001FD12268D30604D5532302A95B18202114
:10AB40001970130704D5532302A95B182B21197020
:10AB500033782A2B16D0350000210A20E3682A78A2
:10AB60006E1C303A092A4ED9002918D010E0013560
:10AB7000B1E7414B2268C01A01238340134323608D
:10AB80002E00CEE7059B191D1B680591002B01DBEC
:10AB9000099304E05B42E3600223134323602B78B4
:10ABA0002E2B0AD16B782A2B35D1059B02351A1D25
:10ABB0001B680592002B2BDB0793304E297803226C
:10ABC0003000FFF7DBFB002806D04023801B8340CA
:10ABD00022680135134323602978062228486E1C19
:10ABE0002176FFF7CBFB00283CD0264B002B25D14C
:10ABF0000722059B07339343083305936369039A40
:10AC00009B18636166E7434301219B183500A6E763
:10AC100001235B42D0E700230A201A00013563605C
:10AC200029786E1C3039092903D9002BC5D0079229
:10AC3000C3E74243012352183500F1E705AB009307
:10AC40003A00114B21000298FEF714F90390039B80
:10AC50000133D3D1BB890B985B0600D42FE70120C9
:10AC600040422CE705AB00933A00074B21000298C5
:10AC7000FEF7BAFBEAE7C04624C100002AC1000083
:10AC80002EC10000758E0000CDA900000B1F1B68AF
:10AC9000181F002B01DA0B58C018704770B5002838
:10ACA0002DD0C317C5185D40C40F2800FDF704FF61
:10ACB000154B1B1A5B055B0D0A2815DD0B3885400B
:10ACC00000222D032D0B002110002D030A0D2D0B4A
:10ACD00012052A430D4D1B052A4013435B00E40770
:10ACE0005B082343190070BD020029001532914012
:10ACF0000A000B21081AC5402D032D0BE3E70024A1
:10AD0000002300250022DEE71E040000FFFF0F8065
:10AD1000044A1368002B00D1034B18181060180068
:10AD20007047C046641000206C100020F8B5C04683
:10AD3000F8BC08BC9E467047F8B5C046F8BC08BCD5
:10AD40009E4670472500252E3166E900252E316686
:10AD50007700506C7573004D6F696E73000A426F17
:10AD6000786D6F644669726D7761726500C389633F
:10AD7000686563206465206C27696E697469616C1D
:10AD800069736174696F6E206465206C27C3A96361
:10AD900072616E204F4C454400000000000000002E
:10ADA00000000000432600002B240000F7230000D1
:10ADB000552400004F240000F52600006724000001
:10ADC0008124000085250000DD240000C12400004E
:10ADD000072400008F2600001F240000B325000078
:10ADE000FB230000572400005F2400000000000047
:10ADF000003E5B4F5B3E3E6B4F6B3E1C3E7C3E1C01
:10AE0000183C7E3C181C577D571C1C5E7F5E1C0046
:10AE1000183C1800FFE7C3E7FF0018241800FFE7FD
:10AE2000DBE7FF30483A060E2629792926407F05C0
:10AE30000507407F05253F5A3CE73C5A7F3E1C1CD6
:10AE400008081C1C3E7F14227F22145F5F005F5F96
:10AE500006097F017F006689956A60606060609482
:10AE6000A2FFA29408047E040810207E2010080887
:10AE70002A1C08081C2A08081E101010100C1E0C92
:10AE80001E0C30383E3830060E3E0E060000000024
:10AE90000000005F00000007000700147F147F140B
:10AEA000242A7F2A12231308646236495620500050
:10AEB00008070300001C2241000041221C002A1C3C
:10AEC0007F1C2A08083E0808008070300008080827
:10AED0000808000060600020100804023E51494547
:10AEE0003E00427F400072494949462141494D3365
:10AEF0001814127F1027454545393C4A49493141CC
:10AF0000211109073649494936464949291E000099
:10AF100014000000403400000008142241141414EE
:10AF20001414004122140802015909063E415D59DA
:10AF30004E7C1211127C7F494949363E41414122E3
:10AF40007F4141413E7F494949417F090909013E0D
:10AF5000414151737F0808087F00417F4100204034
:10AF6000413F017F081422417F404040407F021C46
:10AF7000027F7F0408107F3E4141413E7F0909095D
:10AF8000063E4151215E7F09192946264949493229
:10AF900003017F01033F4040403F1F2040201F3FEF
:10AFA0004038403F63140814630304780403615974
:10AFB000494D43007F4141410204081020004141B6
:10AFC000417F040201020440404040400003070862
:10AFD0000020545478407F2844443838444444285E
:10AFE000384444287F385454541800087E09021805
:10AFF000A4A49C787F0804047800447D400020408D
:10B00000403D007F1028440000417F40007C0478D0
:10B0100004787C080404783844444438FC18242418
:10B020001818242418FC7C08040408485454542498
:10B0300004043F44243C4040207C1C2040201C3C15
:10B040004030403C44281028444C9090907C44640C
:10B05000544C44000836410000007700000041369F
:10B06000080002010204023C2623263C1EA1A16125
:10B07000123A4040207A3854545559215555794157
:10B080002254547842215554784020545579400C2C
:10B090001E5272123955555559395454545939550F
:10B0A0005454580000457C410002457D4200014552
:10B0B0007C407D1211127DF0282528F07C545545E6
:10B0C000002054547C547C0A097F49324949493252
:10B0D0003A4444443A324A4848303A4141217A3A63
:10B0E00042402078009DA0A07D3D4242423D3D402F
:10B0F00040403D3C24FF2424487E4943662B2FFCDE
:10B100002F2BFF0929F620C0887E0903205454798B
:10B11000410000447D413048484A32384040227A5C
:10B12000007A0A0A727D0D19317D2629292F2826D9
:10B130002929292630484D402038080808080808E1
:10B140000808382F10C8ACBA2F102834FA00007B3A
:10B15000000008142A142222142A1408550055004D
:10B1600055AA55AA55AAFF55FF55FF000000FF003C
:10B17000101010FF00141414FF001010FF00FF1037
:10B1800010F010F0141414FC001414F700FF000069
:10B19000FF00FF1414F404FC141417101F10101FE8
:10B1A000101F1414141F00101010F0000000001FD6
:10B1B000101010101F10101010F010000000FF10E1
:10B1C0001010101010101010FF10000000FF1400DD
:10B1D00000FF00FF00001F10170000FC04F414140F
:10B1E0001710171414F404F40000FF00F7141414DB
:10B1F00014141414F700F7141414171410101F105B
:10B200001F141414F4141010F010F000001F101F7D
:10B210000000001F14000000FC140000F010F010EB
:10B2200010FF10FF141414FF141010101F00000062
:10B2300000F010FFFFFFFFFFF0F0F0F0F0FFFFFF66
:10B240000000000000FFFF0F0F0F0F0F38444438BD
:10B2500044FC4A4A4A347E02020606027E027E020C
:10B2600063554941633844443C04407E201E200617
:10B27000027E020299A5E7A5991C2A492A1C4C7254
:10B2800001724C304A4D4D303048784830BC625ADB
:10B29000463D3E494949007E0101017E2A2A2A2A6B
:10B2A0002A44445F444440514A444040444A514047
:10B2B0000000FF0103E080FF000008086B6B083608
:10B2C00012362436060F090F060000181800000079
:10B2D0001010003040FF0101001F01011E00191D68
:10B2E0001712003C3C3C3C00000000000000000045
:10B2F00000000000212F0000B55C0000F7230000D3
:10B300003D280000AD5B0000052900000729000072
:10B310003129000011290000212900003F280000E8
:10B3200005290000332B0000A72A0000492900004E
:10B3300085290000C12900000D2A0000A92A00006B
:10B34000272A0000010203000000000000000000A6
:10B350005D300000D13000006F3000007930000017
:10B360003D300000DD300000213100005D32000082
:10B370005D3100005B3000005B3000000D320000EA
:10B380005F300000000000000001800000000000AD
:10B390000000000003800000000000000000000723
:10B3A000C000000000000000000007C00000000016
:10B3B00000000000000FC0000000000000000000BE
:10B3C0001FE00000000000000000001FE00000007F
:10B3D0000000000000003FE000000000000000004E
:10B3E000003FF00000000000000000007FF00000BF
:10B3F00000000000001FF87FF000000000000000C7
:10B400003FFE7FF0000000000000003FFF7FF000E3
:10B410000000000000001FFFFBE000000000000033
:10B42000000FFFF9FFC00000000000000FFFF9FF50
:10B43000F800000000000007FFF1FFFF000000001F
:10B44000000003FC73FFFF80000000000001FE3FCE
:10B45000FFFF80000000000000FF1E0FFF00000043
:10B46000000000007FFE1FFC000000000000003F05
:10B47000FFFFF8000000000000000FDFFFE0000009
:10B4800000000000001F19FFC000000000000000C5
:10B490003F3CFF00000000000000007E7CF8000040
:10B4A0000000000000007FFE7C00000000000000A3
:10B4B00000FFFFFC0000000000000000FFFFFE0096
:10B4C00000000000000000FFFFFE00000000000080
:10B4D0000001FFEFFE0000000000000001FFCFFEB2
:10B4E0000000000000000003FF07FE000000000055
:10B4F000000003FC07FE0000000000000003F00352
:10B50000FE00000000000000018000FE00000000BE
:10B510000000000000007E000000000000000000AD
:10B52000003E000000000000000000000C000000D1
:10B53000000000078000FC000003C000000007803E
:10B5400001FC000003C0000000078001FC000003B4
:10B55000C0000000078001E00000001E000000079E
:10B560008001E00000001E007FE3F79FF9FDE7780F
:10B570007BDFC0FFF7FFBFFDFDFF787BDFC0FFF77C
:10B58000FFBFFDFDFF787BDFC0F0F787BC3DE1FF2B
:10B59000787BDE00F0F787BC3DE1F0787BDE0000D1
:10B5A000F787803DE1E0787BDE007FF7879FFDE154
:10B5B000E0787BDE00FFF787BFFDE1E0787BDE000F
:10B5C000F0F787BC3DE1E0787BDE00F0F787BC3D1B
:10B5D000E1E0787BDE00F0F787BC3DE1E0787BDEE0
:10B5E00000FFF7FFBFFDE1E07FFBDFC0FFF7FFBF1C
:10B5F000FDE1E07FFBDFC07CF3F39F3DE1E03E7BBC
:10B60000CFC00000000000000000000000FFFFFFAE
:10B61000FFFFFFFFFFFFFFC0FFFFFFFFFD68DB1124
:10B620001A31C0FFFFFFFFFD2B5AFB6AEFC0FFFF7F
:10B63000FFFFFD4B5B3B1A33C0FFFFFFFFFD6B5B62
:10B64000DB6AFDC000006000000000000000000098
:10B650000000000000E0000000000000000000000A
:10B6600000000001E00000000000000000000000F9
:10B67000000001F0000000000000000000000000D9
:10B680000003F000000000000000000000000000C7
:10B6900007F00000000000000000000000000007AC
:10B6A000F8000000000000000000000000000FF89B
:10B6B00000000003C0007E000001E0007F0FF800E2
:10B6C000000003C000FE000001E000FFEFF80000F2
:10B6D0000003C000FE000001E000FFFFF8000000D2
:10B6E00003C000F00000000F007FFE7FC0000003D9
:10B6F000C000F00000000F003FFE7FF83FF1FBCFDD
:10B70000FCFEF3BC3DEFE01FFE7FFF7FFBFFDFFE93
:10B71000FEFFBC3DEFE01FC6FFFF7FFBFFDFFEFE2D
:10B72000FFBC3DEFE00FE3C7FE787BC3DE1EF0FFFA
:10B73000BC3DEF0007FF87FC787BC3DE1EF0F83CC2
:10B740003DEF0001FFFFF0007BC3C01EF0F03C3D69
:10B75000EF0001F37FE03FFBC3CFFEF0F03C3DEF95
:10B760000003E33F807FFBC3DFFEF0F03C3DEF00D2
:10B7700007E73C00787BC3DE1EF0F03C3DEF00079E
:10B78000FFBE00787BC3DE1EF0F03C3DEF0007FFFC
:10B79000FE00787BC3DE1EF0F03C3DEF000FFFFEA5
:10B7A000007FFBFFDFFEF0F03FFDEFE00FFFFF004B
:10B7B0007FFBFFDFFEF0F03FFDEFE00FF9FF003E03
:10B7C00079F9CF9EF0F01F3DE7E01FF1FF00000088
:10B7D0000000000000000000001F80FF007FFFFF4E
:10B7E000FFFFFFFFFFFFFFE01C007F007FFFFFFF69
:10B7F000FEB46D888D18E000001F007FFFFFFFFE84
:10B8000095AD7DB577E000000F007FFFFFFFFEA53F
:10B81000AD9D8D19E0000006007FFFFFFFFEB5AD76
:10B82000EDB57EE00000000000000000212F0000C8
:10B83000B55C0000F72300003D280000F132000055
:10B840000529000007290000312900001129000006
:10B85000212900003F28000005290000332B0000AB
:10B86000BF340000473B0000F93A0000C129000046
:10B870000D2A0000A92A0000272A00000080C0E04D
:10B88000F0F8FCFE000103070F1F3F7FAED580A834
:10B89000D300408D2000A1C8DB40A4A62EAF22001B
:10B8A000FF210000000000000B000000020000006B
:10B8B00004000000FF00FFFFFFFF0B00000000007E
:10B8C0000A0000000200000004000000FF00FFFF6B
:10B8D000FFFF0A00000000000E000000080000004A
:10B8E00004000000FF00FFFFFFFF0E00000000004B
:10B8F00009000000040000001C000000FF0001001F
:10B900000100090000000000080000000400000021
:10B910001C000000FF0000000000100000000000FC
:10B920000F000000040000001C000000FF000103E5
:10B9300001030F00000000001400000005000000DB
:10B940002C000000FF0002000200040000000000C4
:10B9500015000000050000002C000000FF0003009F
:10B9600003000500000000000600000004000000C5
:10B970001C000000FF0000010001060000000000A4
:10B9800007000000040000001C000000FF0001018F
:10B990000101070000000000120000000400000088
:10B9A0001C000000FF000003000302000000000074
:10B9B00010000000040000001C000000FF00000256
:10B9C000000200000000000013000000050000005D
:10B9D0002C000000FF000300030003000000000033
:10B9E00011000000040000001C000000FF00010224
:10B9F0000102010000000000020000000100000040
:10BA0000020000000000FFFFFFFF02000100000035
:10BA100008000000010000001800000002000004FF
:10BA200000040800010000000900000001000000FF
:10BA300018000000030001040104090000000000D8
:10BA40000400000001000000000000000400FFFFEF
:10BA5000FFFF0400000000000500000001000000DE
:10BA6000000000000500FFFFFFFF050001000000CF
:10BA70000200000001000000000000000A00FFFFBB
:10BA8000FFFF02000000000016000000020000009E
:10BA900004000000FF00FFFFFFFF060000000000A1
:10BAA000170000000200000004000000FF00FFFF7C
:10BAB000FFFF0700000000000C0000000300000072
:10BAC00004000000FF00FFFFFFFF0C00010000006A
:10BAD0000A0000000300000004000000FF00FFFF58
:10BAE000FFFF0A00010000000B000000030000003F
:10BAF00004000000FF00FFFFFFFF0B00010000003B
:10BB0000030000000B00000004000000FF00FFFF26
:10BB1000FFFFFF00000000001B0000000B00000002
:10BB200004000000FF00FFFFFFFFFF000000000017
:10BB30001C0000000600000000000000FF00FFFFE6
:10BB4000FFFFFF00000000001800000006000000DA
:10BB500000000000FF00FFFFFFFFFF0000000000EB
:10BB6000190000000600000000000000FF00FFFFB9
:10BB7000FFFFFF00010000001600000003000000AE
:10BB800000000000FF00FFFFFFFFFF0001000000BA
:10BB9000170000000300000000000000FF00FFFF8E
:10BBA000FFFFFF0000000000160000000200000080
:10BBB00000000000FF00FFFFFFFFFF00000000008B
:10BBC000170000000200000000000000FF00FFFF5F
:10BBD000FFFFFF0000000000130000000200000053
:10BBE00000000000FF00FFFFFFFFFF00000000005B
:10BBF000100000000200000000000000FF00FFFF36
:10BC0000FFFFFF0000000000120000000200000023
:10BC100000000000FF00FFFFFFFFFF00000000002A
:10BC2000110000000200000000000000FF00FFFF04
:10BC3000FFFFFF00000000000D00000004000000F6
:10BC40000C000000FF000100FFFF0D0000000000DD
:10BC500015000000050000000C000000FF000300BC
:10BC6000FFFFFF00000000000600000004000000CD
:10BC70000C000000FF000001FFFFFF0000000000BB
:10BC800007000000040000000C000000FF0001019C
:10BC9000FFFFFF00000000000300000001000000A3
:10BCA00002000000FF00FFFFFFFFFF000000000098
:10BCB0000200000001000000020000001400FFFF6D
:10BCC000FFFF0200000000001E0000000400000052
:10BCD00006000000FF00FFFF00010A000000000056
:10BCE0001F0000000400000006000000FF00FFFF2E
:10BCF00001010B0000C2010000000800000000006C
:10BD000000000000CD43000005460000C9430000CC
:10BD1000E9450000C94500004146000025460000F5
:10BD2000C5430000C7430000B94500006546000058
:10BD3000F7450000E1430000494300000D450000C5
:10BD400071430000F0FFFFFF00000000A945000064
:10BD5000FD4400008B460000B543000000000000D9
:10BD600000000000CD4800004F550000275500009E
:10BD700033550000354700003747000025480000D4
:10BD800041726475696E6F205A65726F000004031A
:10BD9000090441726475696E6F204C4C43001201B6
:10BDA0000002EF02014041234D8000010102030126
:10BDB0000000000000000000DD5A0000B55C00003B
:10BDC00067570000B357000061570000795B00001F
:10BDD0007757000051570000115800008F5700009E
:10BDE0004D5700000D0A00001A001A001B001B002E
:10BDF0001C001C001D001D00207700009275000033
:10BE0000D67500003A750000D6750000C6760000B1
:10BE1000D67500003A75000092750000927500001A
:10BE2000C67600003A7500003275000032750000D9
:10BE300032750000D4760000487E00004A7D000084
:10BE40004A7D000068800000447D0000447D0000C1
:10BE50005080000068800000447D00005080000099
:10BE6000447D0000688000005E8000005E8000006D
:10BE70005E8000006C8000004300504F5349580022
:10BE80002E00494E4600696E66004E414E006E61BE
:10BE90006E00300030313233343536373839414274
:10BEA0004344454600303132333435363738396112
:10BEB000626364656600002020202020202020206E
:10BEC000282828282820202020202020202020204A
:10BED000202020202020208810101010101010107A
:10BEE00010101010101010040404040404040404BE
:10BEF0000410101010101010414141414141010146
:10BF00000101010101010101010101010101010121
:10BF1000010110101010101042424242424202022F
:10BF200002020202020202020202020202020202F1
:10BF3000020210101010200000000000000000009D
:10BF400000000000000000000000000000000000F1
:10BF500000000000000000000000000000000000E1
:10BF600000000000000000000000000000000000D1
:10BF700000000000000000000000000000000000C1
:10BF800000000000000000000000000000000000B1
:10BF900000000000000000000000000000000000A1
:10BFA0000000000000000000000000000000000091
:10BFB00000000000000000496E66696E6974790037
:10BFC0004E614E0000000000000000000000000074
:10BFD0000000000000000000000000000000000061
:10BFE0000000000000000000000000000000000051
:10BFF0000000000000000000000000000000000041
:10C000000000000000000000000000000000000030
:10C010000000000000000000000000000000000020
:10C0200000000000000000000080E03779C34143B9
:10C03000176E05B5B5B89346F5F93FE9034F384D8E
:10C04000321D30F94877825A3CBF737FDD4F15753A
:10C05000000000000000F03F00000000000024404D
:10C0600000000000000059400000000000408F4028
:10C07000000000000088C34000000000006AF84093
:10C080000000000080842E4100000000D0126341B7
:10C090000000000084D797410000000065CDCD412D
:10C0A000000000205FA00242000000E8764837420E
:10C0B000000000A2941A6D42000040E59C30A242AC
:10C0C0000000901EC4BCD64200003426F56B0C4321
:10C0D0000080E03779C3414300A0D88557347643C8
:10C0E00000C84E676DC1AB43003D9160E458E14329
:10C0F000408CB5781DAF154450EFE2D6E41A4B449E
:10C1000092D54D06CFF08044F64AE1C7022DB544E2
:10C11000B49DD9794378EA44050000001900000075
:10C120007D000000232D302B2000686C4C006566DC
:0CC13000674546470000000000000000CA
:10C13C00000000006400000066668E41CDCC8C3F90
:10C14C00002000420024004200280042002C004243
:10C15C000030004200340042FFFFFFFFFFFFFFFFF3
:10C16C0040420F0008000000FFFFFFFF40000020CE
:10C17C0000000000E4BF000004C00000C4BF0000C9
:10C18C0000000000000000000000000000000000A3
:10C19C000000000000000000000000000000000093
:10C1AC000000000000000000000000000000000083
:10C1BC000000000000000000000000000000000073
:10C1CC000000000000000000000000000000000063
:10C1DC004300000000000000000000000000000010
:10C1EC000000000000000000000000000000000043
:10C1FC0043000000000000000000000000000000F0
:10C20C000000000000000000000000000000000022
:10C21C0043000000000000000000000000000000CF
:10C22C000000000000000000000000000000000002
:10C23C0043000000000000000000000000000000AF
:10C24C0000000000000000000000000000000000E2
:10C25C00430000000000000000000000000000008F
:10C26C0000000000000000000000000000000000C2
:10C27C00430000000000000000000000000000006F
:10C28C0000000000000000000000000000000000A2
:10C29C00430000000000000000000000000000004F
:10C2AC000000000000000000000000000000000082
:10C2BC007F960000818B000000000000B6BE0000DD
:10C2CC0080BE0000E6BD0000E6BD0000E6BD00003B
:10C2DC00E6BD0000E6BD0000E6BD0000E6BD0000C6
:10C2EC00E6BD0000E6BD0000FFFFFFFFFFFFFFFF04
:10C2FC00FFFFFFFFFFFF00000100415343494900CE
:10C30C000000000000000000000000000000000021
:10C31C0000000000000000000000415343494900A8
:10C32C000000000000000000000000000000000001
:10C33C00000000000000000000000000DD200000F4
:10C34C00852200002528000095320000153D0000D4
:10C35C0021470000B1550000B5200000000000008E
:0400000300005FADED
:00000001FF
